:020000040800F2
:104C0000401F00205D4E0008C9800008AD65000807
:104C10000000000000000000000000000000000094
:104C2000000000000000000000000000454D0008EA
:104C30000000000000000000E94D0008494E000897
:104C40006F4E00086F4E0008E19100086F4E00089B
:104C50006F4E00085D590008ED5900086F4E0008BE
:104C60006F4E00086F4E00080958000811580008E0
:104C70006F4E00086F4E00086F4E00086F4E000820
:104C80006F4E00086F4E0008000000006F4E0008D5
:104C90006F4E00086F4E00086F4E00086F4E000800
:104CA0006F4E00086F4E00086F4E00080DA10008FF
:104CB000C1A10008000000006F4E000800000000C5
:104CC0000348854600F006FA00480047C9B30008CB
:104CD000401F002080F309887047EFF30980704778
:104CE000684680F3098806480078C00703D103208E
:104CF00080F314887047022080F314887047000006
:104D0000A0BC0008064B9C46EFF305831B0605D1AB
:104D1000EFF31483DB0701D000DF7047604700002A
:104D200071B40008064B9C46EFF305831B0605D1C2
:104D3000EFF31483DB0701D000DF7047604700000A
:104D40001DB60008EFF309808169891E09780029E2
:104D500033D1A6461FC8A4467446E0471F4B06CB76
:104D6000914224D0083B002910D00CB420310123FB
:104D70008B71EFF30983203BCB60F0C344464D4673
:104D800056465F46F0C306F04FFE0CBC1A60203258
:104D9000D3681033F0CBA046A946B246BB4683F396
:104DA0000988203BF0CB9079002803D05079EFF3AD
:104DB000098318600223DB43184710B5084A1268BC
:104DC000914209D8074C89006458A6461FC8A446DA
:104DD000F047EFF309840FC410BD000070010020FC
:104DE000085200080852000806F0F0FC154B06CBEC
:104DF000914223D0083B0CB4203100238B71EFF398
:104E00000983203BCB60F0C344464D4656465F467F
:104E1000F0C306F009FE0CBC1A602032D3681033D0
:104E2000F0CBA046A946B246BB4683F30988203B97
:104E3000F0CB9079002801D0507918610223DB4330
:104E4000184700007001002006F0A6FECEE7000023
:104E500006F0F6FA06F0A0FEC8E700000448804716
:104E600004480047FEE7FEE7FEE7FEE7FEE7FEE751
:104E7000D19C0008C14C000830B50B46014600200B
:104E80002022012409E00D46D5409D4205D31D4650
:104E90009540491B2546954040191546521E002D48
:104EA000F1DC30BD70B500242546002801DA01246C
:104EB0004042002901DA01254942FFF7DDFFAC42FB
:104EC00000D04042002C00D0494270BD03460B4345
:104ED0009B0703D009E008C9121F08C0042AFAD2B0
:104EE00003E00B780370401C491C521EF9D2704736
:104EF000D2B201E00270401C491EFBD27047002272
:104F0000F6E710B513460A4604461946FFF7F0FFC8
:104F1000204610BD421E5378521C002BFBD10B784B
:104F20001370491C521C002BF9D1704730B505464F
:104F30002A460B4610781C78521C5B1C002801D0B6
:104F4000A042F7D0002C03D0002802D06D1CEFE760
:104F5000284630BD10B5044605E00B780370401CB0
:104F6000002B00D0491C521EF7D2204610BD421C17
:104F70000178401C0029FBD1801A704710B500222F
:104F800000E0521C835C8C5CA34201D1002BF8D161
:104F9000D8B2E1B2401A10BD03460A780270401C34
:104FA000491C002AF9D1184670470321001D401EF4
:104FB000037812021A43491EF9D51046704703467A
:104FC00003220870000A491C521EFAD51846704781
:104FD00070B5064605F066FF046805460A22002102
:104FE000304600F03FF82C6070BD70B5064605F005
:104FF00059FF046805460A220021304600F032F8C5
:105000002C6070BDF0B51FB40646002082B0054686
:105010004024019100901BE0019922460F46304642
:1050200000F07AF8049A059B801A994110D3104633
:105030001946224600F060F8361A8F410197224641
:1050400001200021009F00F057F838184D410090D2
:105050002046641E0028DFDC019B0098294632466A
:1050600007B0F0BDF7B5009C0F4600262578641CFC
:10507000002D05D000F062F80068405DC007F5D152
:105080002B2D02D02D2D18D0641E39462046029AB1
:1050900000F058F8002F04D03968A14201D10099DE
:1050A00039607105022400290BDA4042002803DD33
:1050B00005F0F8FE0460A007FEBD01208002064353
:1050C000E3E70028F8DA05F0EDFE04600048FEBDD5
:1050D000FFFFFF7F064C0125064E05E0E36807CC85
:1050E0002B430C3C98471034B442F7D3FFF7ECFD48
:1050F000D0BE0008F0BE000810B5202A04DB01462F
:10510000203A9140002010BD914020239C1A034674
:10511000E3401943904010BD10B5202A04DB084637
:10512000203AD040002110BD0B46D340D04020246F
:10513000A21A91400843194610BD0000004870476C
:105140008CBE0008F7B582B0029C00272078641C52
:1051500015460197302802D0002D15D015E0207893
:105160000127641C782804D0582802D0002D09D0CB
:105170000BE0002D01D0102D07D10027102520783D
:10518000641C02E0082500E00A250026009610E0D5
:105190000099012769430818020C294680B271431F
:1051A00000908E183804864201D3012001902078A7
:1051B000641C294600F019F80028E9DA0398002851
:1051C00005D0002F01D0641E00E0029C046001980D
:1051D000002806D005F066FE02210160C81E05B059
:1051E000F0BD009930040843F9E73A2800D230387E
:1051F000202302469A43412A01D310463738884279
:1052000001D30020C04370470000000010B50B46DA
:105210000021846A1C43846200BF0C46144321466B
:10522000416110BD002904D0826801231A438260C5
:1052300003E0826802231A4382607047002904D089
:10524000C26801231A43C26003E0C26852085200D8
:10525000C2607047C26802239A43C260C2680A43B0
:10526000C260704710B504460548844207D1012149
:10527000401503F0B9FE0021601503F0B5FE10BD26
:105280000024014000B589B00121480203F09CFED2
:1052900001200790032108A801700021C17007A90F
:1052A0000920C00600F0C6FE1F48FFF7DBFF1F48BD
:1052B00003F04EFE02211C48FFF7CCFF00211A48E4
:1052C000FFF7BCFF01A800F08AF800200190002140
:1052D00068460172002003900590069001A91248CB
:1052E00000F062F8052201210F48FFF78FFF0E48FA
:1052F00000F020F801210C48FFF7A0FF01210A4827
:10530000FFF790FF00BF0A49074800F035F8002872
:10531000F9D000200449886201208862084600F024
:1053200059F809B000BD0000002401400040000110
:105330000100000130B501460020002200238C68E6
:105340000125ED072C438C6000BF8C68E30FDB0761
:10535000521C0F242403A24201D0002BF5D18C68EB
:10536000E40FE407002C01D1086C00E0002030BD00
:105370000146086C80B2704730B502460020002319
:10538000012424060C40002C05D0946801252D062C
:10539000AC43234600E013681C460C40002C01D0AF
:1053A000012000E0002030BD10B50022C268084B8B
:1053B0001A400C7964030B6823438C682343CC6840
:1053C00023430C6923434C6923431A43C26010BD35
:1053D00003D2FFFF816804221143816070470021DE
:1053E000016001718160C16001614161704700002D
:1053F0001CB5002168460171032141710121C17171
:105400000803009069460920C00600F013FE012041
:10541000C002009069460920C00600F00BFE012082
:10542000C003009069460920C00600F003FE082072
:1054300000906946264800F0FDFD01216846017193
:1054400000218171C171102000906946204800F050
:10545000F1FD4020009069461D4800F0EBFD012061
:105460000003009069461A4800F0E4FD0120400363
:1054700000906946164800F0DDFD20200090694646
:10548000134800F0D7FD012000906946104800F055
:10549000D1FD01200E498861022000906946092053
:1054A000C00600F0C7FD02200A4908818020009054
:1054B0000221684601710121C1716946044800F06A
:1054C000B9FD02220721024800F0FCFD1CBD0000CE
:1054D000000400482000004810B5002400BF0AE086
:1054E000A0000A4940180068A1000122520789184B
:1054F0000860601CC4B2302CF2DB0121084603F0C6
:1055000063FD032004F0F4F810BD0000004C000817
:10551000F7B50B461446009D002C12D10CE017077E
:105520003F0F1611304600F023F818705B1C384608
:1055300000F01EF818705B1C2A786D1C002AEED152
:1055400013E010E02A786D1C17073F0F1611304644
:1055500000F00EF818705B1C384600F009F818705F
:105560005B1C601EC4B2002CECD100201870FEBD84
:10557000002805DB092803DC01463031C8B208E009
:105580000A2805DB0F2803DC01465731C8B200E0CA
:10559000FF20704710B50446204600F007F810BD04
:1055A00000200149087070472501002070B50546AC
:1055B0000AA1284602F008FB00280ED1E81DFFF7DB
:1055C00007FDC4B2002C08DB642C06DA054884729F
:1055D00001460D312046FFF7F2FC70BD2B434353CB
:1055E000513A0000F819002010B50446244800780C
:1055F00000280DD12348006823490968884200D259
:1056000010BD204800682049086001201C4908702E
:10561000FF204130844215DA1CA1002004F070FA0A
:105620001E484079012806D101221DA1032001F066
:105630002DFD02F001FA00201849487104F02CFBFE
:1056400000BFFEE7FF205530844212DA0D480068A3
:105650000D490968884210D90A4800687D2109016E
:10566000401809490860012212A1032001F00EFD33
:1056700003E0044800680449086000BFC0E7000078
:10568000540100207801002050010020565F4C6F2B
:1056900077205077724F66660D0A0000BC1100201B
:1056A0003445344638423533373335313341363774
:1056B0000000000046373842343535313335373550
:1056C0000000000010B50446002C04D0012C31D09D
:1056D000022C76D133E03CA1002004F011FA3D48C1
:1056E000047000223C493D4804F014FE01223C496C
:1056F0003A4804F00FFE01228021384804F0CFFD23
:1057000001224021354804F0CAFD002232493548C3
:1057100004F000FE01223249324804F0FBFD002271
:105720008021304804F0BBFD012240212D4804F0C7
:10573000B6FD46E02CA1002004F0E2F941E02DA1E5
:10574000002004F0DDF92348047001222249234897
:1057500004F0E0FD00222249204804F0DBFD002295
:1057600080211E4804F09BFD002240211B4804F0CC
:1057700096FD0021234800F05BF8002121481430F9
:1057800000F056F801221449164804F0C3FD002227
:105790001349144804F0BEFD00228021114804F092
:1057A0007EFD002240210F4804F079FD00211548BC
:1057B000283000F03DF8002112483C3000F038F865
:1057C00000BF00BF10BD0000434F4D2D3E4D43555F
:1057D000210D0A002C0100200501050000380140C0
:1057E0000401040000440040434F4D2D3E475053F8
:1057F000210D0A00434F4D2D3E4D6F64656D210D07
:105800000A0000001C00024010B504F0C1FC10BDED
:1058100010B504F013FD10BD014948607047000049
:10582000000002400149486070470000000002404B
:10583000002904D0026801231A43026003E00268D1
:10584000014B1A4002607047FEFF00000168254AC4
:10585000114001600021016041608160C160224906
:10586000884208D12049083949680F2211431E4A4D
:10587000083A516035E01C491431884208D11A4970
:1058800008394968F0221143174A083A516028E064
:1058900015492831884209D11349083949680F222E
:1058A00012021143104A083A51601AE00E493C3185
:1058B000884209D10C49083949680F221203114363
:1058C000094A083A51600CE007495031884208D132
:1058D0000549083949680F2212041143024A083A5F
:1058E00051607047FEFF00000800024001460020A2
:1058F000044A12680A40002A01D0012000E000207A
:105900007047000000000240002A03D003680B43E8
:10591000036002E003688B430360704710B5002208
:1059200002680D4B1A400C6A8B6823430C692343B1
:105930004C6923438C692343CC6923434C6A23433A
:105940008C6A23431A430260CB6843600B68836010
:105950004B68C36010BD00000F80FFFF10B5022030
:1059600000F092F8002815D01C48008A0221084057
:10597000002806D01A480078012108431849087009
:1059800005E01748007840084000154908700220DB
:1059900000F074F812480078002802D0032817D1CC
:1059A0000AE010480078012802D10F49C87102E0CE
:1059B00002200D49C8710BE00A480078012803D184
:1059C00002200949C87102E001200749C87100BFDF
:1059D00000BF034800780349087010BD0004004868
:1059E000C0000020C10000202F08002010B50420B6
:1059F00000F04AF8002815D01C48008A042108400D
:105A0000002806D01A480078022108431849087077
:105A100005E01748007802218843154908700420E2
:105A200000F02CF812480078002802D0032817D183
:105A30000AE010480078012802D10F49C87102E03D
:105A400002200D49C8710BE00A480078012803D1F3
:105A500002200949C87102E001200749C87100BF4E
:105A600000BF034800780349087010BD00040048D7
:105A7000C0000020C10000202F080020014948611B
:105A80007047000000040140014600200022074B3F
:105A90001B680B401A46054B5B690B40002B03D07B
:105AA000002A01D0012000E00020704700040140DE
:105AB000002120498279002A35D00A4612680368FD
:105AC0009A430B461A600A46526803689A430B468B
:105AD0005A60027951180A6803681A430A60154A25
:105AE000926803689A43134B9A601A46D268036817
:105AF0009A43104BDA604279102A0CD11A46926808
:105B000003681A430B4B9A601A46D26803681A431B
:105B1000084BDA600DE00749427951180A680368BA
:105B20001A430A6005E0027951180A6803689A432B
:105B30000A607047000401401FB5002168460173E8
:105B4000032141730021C1730620029002A90E486F
:105B500000F070FA0220FFF791FF0420FFF78EFF9C
:105B60000221012003F0A4FD0121084603F0A0FD5D
:105B70000620009000216846017110214171012129
:105B80008171FFF795FF1FBD0004004800B589B083
:105B90006B48C079002879D0012802D0022876D13C
:105BA00064E067480078C007C00F002804D064484C
:105BB000007A401C624908726148007802218843DB
:105BC0005F4908705F48C078002808D15D480079B7
:105BD000002804D108464078401C4870A9E0012004
:105BE000594908815748C07800280FD002205549EC
:105BF000C8700120544908810022114653A001F0C9
:105C00004DFF57A1002003F07BFF2EE04D480079A7
:105C100000282AD002204B490871534840890028A7
:105C200007D151498881002250A1012001F02EFAAC
:105C30000AE04D48828955A101A805F011F900221A
:105C4000114601A801F02AFF47488089401C4649B7
:105C50008881084680894989884202DB00204249C0
:105C6000888150A1002003F04BFF62E000203449FE
:105C700008723448C07800280AD1324800790028D8
:105C800006D108468078401C887052E04FE04FE013
:105C90002C48C07800280FD002202A49C870012063
:105CA000294908810022114641A001F0F7FE45A1D3
:105CB000002003F025FF39E022480079002835D084
:105CC00002202049087128484089002805D1012276
:105CD0003EA1032001F0DAF90EE02348828943A1B6
:105CE00001A805F0BDF80022114601A801F0D6FE7A
:105CF00001A9002003F004FF1B488089002805DD6E
:105D000019488089401E184988810BE0164840894F
:105D1000002802D11449888104E013484089401EBC
:105D20001149888137A1002003F0EAFE01E000E07C
:105D300000BF00BF00200249C87109B000BD0000CB
:105D40002F080020E81200202004004841542B5066
:105D50004F433D31303030303030370D0A000000D5
:105D60005B472B2B5D0D0A00BC11002043454445C9
:105D70004336453443424643423343394434423147
:105D800044344441434644460000000041542B50F3
:105D90004F433D3130303030303231253034780DA2
:105DA0000A0000005B557365722B2B5D000000003C
:105DB00041542B504F433D31303030303030380D6E
:105DC0000A0000005B472D2D5D0D0A004530363579
:105DD000373635313833354231303632353835346F
:105DE00032383537424637450000000041542B50C9
:105DF0004F433D3130303030303231253034780D42
:105E0000000000005B552D2D5D00000080B51F488F
:105E10000078400840001D49087001201C49088195
:105E20000A219320C00003F085FC1420194FBC46C2
:105E300000DF0120164908810A21174803F07AFC87
:105E40001420BC4600DF0120114908810A2193205B
:105E5000C00003F06FFC01201049087004F000FB43
:105E6000012000F0B1FE082003F0C4FC0CA10020CA
:105E700003F046FE0548007802218843801C034950
:105E8000087020200249088180BD0000F819002018
:105E900020040048C5B500086E030000000900207A
:105EA00047545F4D6F64650D0A0000000149C860EA
:105EB000704700000020024030B5044604250B2046
:105EC000000400F07BF80546042D17D10C4800694A
:105ED000022108430A4908610846446100694021DB
:105EE0000843074908610B20000400F067F80546E5
:105EF000034800690221884301490861284630BDF2
:105F00000020024004200D49C968C907C90F0029B3
:105F100001D0012010E00949C96810221140002970
:105F200001D0022008E00549C96804221140002977
:105F300001D0032000E00420704700000020024050
:105F40000348006980210843014908617047000047
:105F50000020024070B504460D4604260B200004C4
:105F600000F02CF80646042E11D10A4800690121E0
:105F700008430849086125800B20000400F01EF842
:105F8000064604480069400840000249086130465E
:105F900070BD0000002002400548006980210840D3
:105FA000002804D00348024948600348486070470D
:105FB0000020024023016745AB89EFCD10B50346B1
:105FC0000424FFF79FFF044603E0FFF79BFF04460E
:105FD0005B1E012C01D1002BF7D1002B00D1052431
:105FE000204610BD1CB50320694608710C4800907E
:105FF0000920C00600F01EF869460A4800F01AF8A9
:106000006946094800F016F86946084800F012F899
:106010006946074800F00EF8002002F0FFFF1CBDA3
:10602000FFFF00000004004800080048000C004882
:1060300000140048F0B50A4600210023002400BFE8
:106040003DE001258D402B4615681D402C469C42A5
:1060500034D11579012D02D01579022D16D185681C
:106060004F000326BE40B543856055794E00B540CC
:10607000866835438560858801268E40B5438580D6
:10608000858896798E40B6B23543858005684F0085
:106090000326BE40B543056015794E00B54006683D
:1060A00035430560C5684F000326BE40B543C56053
:1060B000D5794E00B540C6683543C560491C1029E6
:1060C000BFD3F0BDF0B5002300244D07EE0E1546FA
:1060D000B5402B46CD10AE0005462035AD594E07D4
:1060E000F70E0F26BE40B543CE10B6000746203748
:1060F000BD51CD10AE003D46AD591D432C46CD10CF
:10610000AD003E467451F0BD20200349088100BF18
:1061100000F07CFAFCE7000020040048F7B58CB0E2
:1061200032490D98884202D200200FB0F0BD0E987F
:10613000FEF71DFF07460E2F03D00F2F01D00020C2
:10614000F3E72BA109A80D9A04F08AFE09A8FEF72F
:106150000EFF009000253C460A3C05E00E98005DCD
:1061600005A948556D1C641CBC42F7DB00260020C5
:106170000190002408E009A8005D464005A8005DE4
:10618000019948400190641C0A2CF4DB01984640B8
:106190001948805D019000240DE009A8005D019977
:1061A0004840064605A8005D704002A908551248FF
:1061B000805D0190641C0A2CEFDB002504240EE0B6
:1061C00002A9085D0A21FEF76DFE0C9841550C9856
:1061D000405D3030C1B20C9841556D1C641C0A2CD6
:1061E000EEDB00210C98817101209EE72058F20817
:1061F000253031306C750000B8BC000810B53E4841
:106200000078401CC0B23C490870012801DD002024
:10621000087039480078002804D100F0BBFC3749E9
:10622000088003E000F0B6FC354908803348008858
:1062300033490988884201D0002010BD2F480488C6
:1062400030480088A04211D02E48048000882E4992
:10625000884206D001202D49087000202C49087082
:1062600004E00020294908702A490870274800786E
:10627000002832D0284800788007C00F002813D0AB
:10628000264800782149097888420BD01F480078B9
:10629000224908701B4801881F48C170090A017112
:1062A0000120CAE70020C8E7184800781B49087099
:1062B0001B4800681B49096888420CD811480188AE
:1062C0001548C170090A0171164800686430144904
:1062D00008600120B1E70020AFE7124800681049CC
:1062E00008600E480078002804D000200B49087090
:1062F000FF20A2E70020A0E7120100201A010020E1
:106300001C01002018010020089800001301002043
:1063100011010020100100202F080020140100208E
:106320002001002078010020F7B588B00E4600203B
:1063300007900024009008980078002802D0307858
:10634000002802D100200BB0F0BD0CE00098411CE9
:10635000009101A90F543D2F01D03B2F01D1002006
:10636000F1E7761C641C3778002F01D0142CEDDB8C
:106370003D222046641C01A90A54002008550898B3
:10638000FEF7D4FD05462D1909E029780A98017019
:106390006D1C0A98401C0A900798401C07902878AA
:1063A000202805DD28783B2802D007982828ECDB38
:1063B00000210A9801700798C5E7000070B5042114
:1063C0002B48FEF7D9FF01280BD12948FEF7D0FF53
:1063D0000446642C0BDA2748844208DD0020C043C1
:1063E00070BD2348FEF7F6FF0020C043F8E72248BF
:1063F0000088A04201DD2048048020480088A04297
:1064000001DA1E4804801E48008800191C490880D3
:106410001C480078401C1B490870084600780A2870
:1064200023DB154800881549098840181449098854
:10643000081A1349088013480078811E1048008804
:10644000FEF730FD0E4908800988FF222D325143A6
:106450000846C917090D091809134D0000200949FC
:106460000870074908802846BAE70120C043B7E70B
:1064700000240140FF0F00003601002038010020F9
:106480003A0100203C010020F0B585B005460E46DB
:106490000027142211496846FEF718FD002407E082
:1064A00060006946085AA84200DD03E0601CC4B2DF
:1064B000142CF5D300BF092C02DD0124302703E0A2
:1064C000002C01D1601CC4B23B462246303204A1EC
:1064D000304604F0C5FC05B0F0BD0000B8BD0008B2
:1064E000253032783030333030302530327830302B
:1064F0000000000070B504460D461F2C01DC012C85
:1065000004DA0FA12846FEF747FD18E0192C04DD38
:1065100012A12846FEF740FD11E0112C04DD14A164
:106520002846FEF739FD0AE00A2C04DD15A12846AD
:10653000FEF732FD03E018A12846FEF72DFD70BDE1
:1065400032433030453036353531374644433745B0
:106550004531344646373533000000004531344676
:10656000463735333833384633413546000000006E
:10657000453134464637353330323930324434458C
:106580000000000045313446463735333446353057
:106590003445344600000000453134464637353333
:1065A000383835463331354600000000704700006A
:1065B00010B504460121C80202F0F6FC5D2002F08D
:1065C000EBFD002801D002F01FFD0B4800F032F86F
:1065D000062000F023F8002C04D0FF20000100F07A
:1065E00023F803E0FF202D3000F01EF800F00EF835
:1065F00000F004F810BD00005555000001480249A4
:1066000008607047CCCC00000030004001480249CF
:1066100008607047AAAA00000030004001494860A5
:10662000704700000030004001498860704700005A
:106630000030004001490860704700000030004011
:1066400009480078FF2804DA07480078401C06490A
:10665000087006480078FF2804DA04480078401CD7
:10666000024908707047000010010020110100204D
:1066700010B566480179C278080210436449401891
:1066800000282AD007210903401A08D00121C90295
:10669000401A0CD0FF21C900401A0ED162E05D48BB
:1066A000007802218843801C5A49087000BF59486D
:1066B0000078C007C00F002800D0A3E0564800783B
:1066C00004218843544908700020544988710022ED
:1066D000114653A001F0E2F994E04F48C079052833
:1066E0003BDA4E480078002832D04B480079002829
:1066F0000CD000204849087101224DA1032000F070
:10670000C5FC4EA1002003F0FBF926E04248C0780A
:1067100000280CD101224CA1032000F0B7FC4FA1AE
:10672000002003F0EDF901203B49C87015E03A481C
:10673000C078012811D100203749C87001223CA13E
:10674000032000F0A3FC47A1002003F0D9F904E0E6
:10675000012247A1032000F099FC00202E49C871B6
:1067600048714FE046480078C007C00F00280FD09E
:10677000294800788007800F012802D104F0F0F842
:1067800005E040A1002003F0BBF902F0F5FD10BDCB
:106790001E48007A022813DD39480078C007C00F70
:1067A00000280DD13A480078C007C00F002807DD47
:1067B000FFF72CFB00201849087214490872E6E71D
:1067C0001548007A032812DA1348007A00280ED000
:1067D000124820300078002804D010486030407CF7
:1067E000002802D102F0C8FD01E002F08FFE002077
:1067F00009490872054908720846007840084000B7
:10680000087000BF00BF00BFC1E700002F080020D4
:10681000F8E7FFFF40010020E8120020BC11002033
:1068200041542B504F433D3043303030300D0A003F
:106830003030393046413531000000005B45787416
:10684000555D0D0A0000000041343746433437459A
:106850003039393045393632000000005B456E472B
:106860005D0D0A005B457874475D0D0A000000006D
:106870003241363737423736343639360000000079
:106880000009002054657374313838380D0A00004F
:10689000F819002010B509210148FEF730FB10BDA2
:1068A0002F08002090B589B0002476480179C2787D
:1068B000080210437449401800286BD007210903CF
:1068C000401A08D00121C902401A05D0FF21C90091
:1068D000401A5ED1AEE000BF6C48007804218843C6
:1068E000001D6A4908706748007802218843801CAF
:1068F0006449087066A1002003F002F96348C0787B
:10690000022819D100206149C87001206749088117
:10691000674A68A101A804F0A3FA01226AA1032032
:1069200000F0B4FB0022114601A801F0B7F81420D2
:10693000684FBC4600DF2CE054480079022820D183
:1069400000205249087164484089002805D100227E
:1069500062A1012000F09AFB0EE00A205D4FBC46C8
:1069600000DF534A093A65A101A804F079FA002230
:10697000114601A801F092F865A1002003F0C0F8CB
:1069800007E00120544988710022114664A001F0FB
:1069900085F873E03B480078022188433949087044
:1069A0004D480078002801D109B090BD3748C07922
:1069B00005283EDA3548C079401C3449C87108467C
:1069C000C079052835D10846C078002831D101208A
:1069D000087157A1002003F093F8012256A103206B
:1069E00000F054FB02203B4FBC4600DF57A101A83A
:1069F00004F036FA0022114601A801F04FF801A96F
:106A0000012003F07DF80220BC4600DF002032495F
:106A1000488188810A46173251A101A804F020FA62
:106A200001A9012003F06CF80022114601A801F031
:106A300035F823E01348007840084000401C114915
:106A4000087008460078022188430E4908700F48F4
:106A5000007A092811DA0D48007A401C0B490872A7
:106A60000846007A032802D102F066FD05E00748D7
:106A7000007A092801D102F093FD00BF00BF00BFDA
:106A800092E700002F080020F8E7FFFFE81200203F
:106A90005B4B45595F5050542F4B45595F505054F4
:106AA0005F4D49432050726573735D0020040048B8
:106AB000D812002041542B504F433D3039303030F4
:106AC0003025730D0A000000444238463635353112
:106AD00000000000C5B50008BC1100204345444536
:106AE00043364534434246434233433944344231CA
:106AF00044344441434644460000000041542B5076
:106B00004F433D30413030303025730D0A000000D6
:106B10005B457869745573657253656C5D00000060
:106B200041542B504F433D3042303030300D0A003D
:106B3000456E550D0A000000313036323538353497
:106B400030393930453936320000000041542B507D
:106B50004F433D31303030303032300D0A000000CC
:106B600041542B504F433D30453030303025730D6C
:106B70000A00000010B5FFF741FB041E06D0012CEF
:106B800002D1FFF78FFE01E0FFF772FDFEF7FEFF77
:106B900010BD00000920C006008A1323DB02184044
:106BA00001460448008A082318400246084610435C
:106BB000704700000004004810200249088140206E
:106BC000088170472004004800281FD00021684A2F
:106BD0001160684A1170684A1170684A1170FF218B
:106BE000674A1170674A11700021674A1170674A3D
:106BF0001170674A1170FF21664A1170664A117060
:106C00001021664A11814021118170476449096849
:106C1000574A1268914200D2F7E7614909680A3180
:106C2000534A11605F490978002903D110215B4A5A
:106C3000118149E05C490978002904D11021574AA3
:106C4000203A916140E04E490978564A12789142C3
:106C500005D14C490978544A1278914219D0002143
:106C6000444A1170484A11704E490978444A1170DB
:106C70004D490978434A11704A4909784906090E75
:106C80003E4A11703F4909784900127889183A4AFA
:106C9000117038490978491CC9B2364A1170364A10
:106CA0001278914202DD0021324A1170314909788F
:106CB000324A1278914204DA1021384A203A91611E
:106CC00002E01021354A118138490978002903D1A1
:106CD0004021324A118149E035490978002904D11F
:106CE00040212E4A203A916140E02A4909782F4AF2
:106CF0001278914205D1284909782D4A127891429B
:106D000019D000211B4A11701F4A117027490978B8
:106D1000204A1170264909781F4A117023490978C1
:106D20004906090E1A4A11701B4909784900127860
:106D30008918164A117014490978491CC9B2124AB7
:106D40001170124A1278914202DD00210E4A117030
:106D50000D4909780E4A1278914204DA40210F4A0F
:106D6000203A916102E040210C4A118100BF4CE7BA
:106D700008010020FD000020FE000020FF00002090
:106D80000001002001010020020100200301002079
:106D90000401002005010020060100202004004815
:106DA00078010020F8000020F9000020FA000020FF
:106DB000FB000020BFB521480078002800D1BFBDEE
:106DC000002211461EA000F069FE1E20204FBC4686
:106DD00000DF01201F49C8701F4908811748437808
:106DE0001EA20F21684604F025F8002211466846CD
:106DF00000F054FE11486630FEF7D7F8002806D19F
:106E0000002211460D48801C00F048FE08E00B48A7
:106E10006630FEF7CAF804460022114600F03EFE36
:106E20000022114611A000F039FE0020034908702D
:106E30001E20074FBC4600DF00BFC0E7B0070020A0
:106E400041542B4C53485454535354500D0A000092
:106E5000C5B50008BC1100202004004841542B4C4B
:106E600053485454533D25642C220000220D0A003F
:106E700008B51B216846017001214170817001F045
:106E800025F91C216846017001214170817001F0D3
:106E90001DF90A21684601700021417001218170AD
:106EA00001F014F90B2168460170002141700121A5
:106EB000817001F00BF905216846017000214170D5
:106EC0000121817001F002F906216846017001215B
:106ED0004170817001F0FAF808BD000092B04421C1
:106EE00001A8FEF70CF840A1002002F009FE0A21DB
:106EF0006F20C00002F01EFC02F08AF90A203E4F0B
:106F0000BC4600DF3D48817D427D080210430346B8
:106F10003A4AD21D3AA101A803F0A2FF01A900201C
:106F200002F0EEFD35481D30FEF73FF805462A46D3
:106F300038A101A803F094FF01A9002002F0E0FDB0
:106F40003748007880088000354908700020887133
:106F50000120BC4600DF33A1002002F0D1FD002358
:106F6000344A35493548364FBC4600DF0023354AA0
:106F700035493648BC4600DF0023354A3549364896
:106F8000BC4600DF2FE001201B4FBC4600DF02F0B3
:106F90002BFE03F007FDFFF7EDFD0020FFF714FEC9
:106FA000FFF70CFA0446002C03DD1D484470210A4B
:106FB00081702A4800682A490968884200D212E094
:106FC00026480068643026490860FFF739FB1449F9
:106FD0008B784A781906091411430846FEF704FB1A
:106FE000FFF714FB00BFCEE74D5461736B30207286
:106FF000756E0D0A00000000C5B5000838080020B5
:1070000025735F5625642053746172742E2E2E0DE5
:107010000A00000050534E3A256C750D0A0000001E
:10702000E81200204D5461736B312072756E0D0AA9
:1070300000000000F8150020030001008D7E00080C
:1070400015BC0008F816002003000300F17B0008BF
:107050003007002003800000259F000878010020F1
:107060004801002070B50546002407E0285D0D2882
:1070700002D10020285570BD601C84B22846FDF75F
:1070800076FFA042F2D800BFF5E70000F7B505464D
:1070900016460198FDF76BFF84B2642C00DD642472
:1070A000012E0FD1224610480199FDF70FFF642CE5
:1070B00002DA00210C4801550B4964310020FDF72C
:1070C0007EFF04E0084964310198FDF778FF064827
:1070D000801E45700078401C0349891E08700348D3
:1070E000034FBC4600DFFEBDB2070020E0000020D9
:1070F000A9B9000800B5AFB02FA2642116A803F00B
:1071000099FE3148407C002804D130A116A8FDF733
:1071100001FF16E02C4B113330A2502102A803F0DE
:1071200089FE0022114602A800F0B8FC264B11335C
:1071300030A2502102A803F07DFE02A916A8FDF797
:10714000E9FE16A9002002F0DBFC2BA2642116A8A0
:1071500003F070FE1C4820304078002804D01A4804
:107160002030407C002804D118A116A8FDF7D2FEDB
:107170001CE0154831300346103B22A250210090FC
:1071800002A803F057FE0022114602A800F086FC78
:107190000D4831300346103B20A25021009002A838
:1071A00003F048FE02A916A8FDF7B4FE16A90020B8
:1071B00002F0A6FC2FB000BD5B31315D4163636519
:1071C0007373703A00000000B8080020756E737584
:1071D00070706F72742D456D7074790041542B4D31
:1071E000495050524F46494C453D312C222573227F
:1071F0000D0A0000257300002C4E616D652D506155
:1072000073733A0041545E5050504346473D222527
:1072100073222C222573220D0A00000025732C25D1
:1072200073000000F0B5BFB000255DE032260022FB
:10723000114631A000F032FC4FE050212BA800F0A5
:1072400065FE0446002C44D02FA12BA800F0BCFC06
:10725000002842D02E48FDF7A8FE07463B462C4AA0
:10726000121D2CA11DA803F0FBFD002201A91DA8E1
:10727000FEF74EF901A92EA8013000F0A5FC002868
:1072800025D12348FDF791FE0746214854303B465F
:107290000246503A23A100901DA803F0E1FD002210
:1072A00001A91DA8FEF734F90022114623A000F021
:1072B000F5FB0022114601A800F0F0FB0022114668
:1072C00022A000F0EBFB22A1002002F019FC3FB04D
:1072D000F0BD0120214FBC4600DF3046711ECEB20A
:1072E0000028AAD1681CC5B2032D9FDB1CA1002079
:1072F00002F006FC00BFEAE741542B504F433D30FB
:1073000032303030300D0A002B504F433A303200CB
:107310005508002069703D25733B69643D256C75F7
:107320000000000069703D25733B69643D256C7564
:107330003B7077643D25733B0000000041542B50A7
:107340004F433D3031303030300000000D0A000036
:1073500052737420504F430D0A000000C5B5000859
:10736000504F43206973204F4B0D0A00F0B597B082
:10737000002400201590002640E032201690002CBA
:107380000BD10124002211461EA000F087FB20A291
:107390000A2112A803F04EFD0AE000240022114643
:1073A0001DA000F07BFB1FA20A2112A803F042FDE2
:1073B0001DE0412101A800F0A9FD0546002D12D0D5
:1073C00012A901A800F000FC002810D1E01D01A9BD
:1073D000085C52280BD120460930085C412806D1B0
:1073E000012017B0F0BD0120104FBC4600DF1698F9
:1073F000411EC9B216910028DBD1761C1E2EBCDBC3
:107400000020EEE741542B514350494E3F0D0A00F6
:107410002B514350494E3A0041542B4350494E3F63
:107420000D0A00002B4350494E3A0000C5B5000834
:10743000012000030349886140000249203108818E
:107440007047000000040048F0B5A7B00020269067
:1074500000256DE064260022114639A000F01EFBD5
:1074600061E04121684600F051FD0446002C56D0F1
:1074700036A1684600F0A8FB002854D1152201A9C6
:1074800003313448FDF722FD0020324908750B46D0
:1074900031A2502112A803F0CDFC2E48017910A88A
:1074A00001712C48417910A841710021817111A806
:1074B000FDF78EFD030003F0E7FC0C1007111A2501
:1074C000251B121C08251D2500BF02202649087017
:1074D00026A112A8FDF71EFD19E000BF00BF012084
:1074E0002149087025A112A8FDF714FD0FE000BF87
:1074F00000BF00BF03201C49087024A112A8FDF79B
:1075000009FD04E025A112A8FDF704FD00BF00BF9E
:1075100012A9002002F0F4FA012027B0F0BD0120EA
:10752000224FBC4600DF3046761E002899D16D1CE4
:10753000052D8FDB1EA1002002F0E2FA0020ECE70F
:1075400041542B49434349440D0A00005E534349CB
:10755000443A00001A0800205B30395D4943434932
:10756000443A25735B0000000C0100204348494E5B
:10757000415F554E49434F4D5D0000004348494E21
:10758000415F4D4F42494C455D0000004348494E24
:10759000415F54454C45434F4D5D0000554E4B4EA9
:1075A0004F572D49434349445D000000C5B50008CD
:1075B0005B30395D47657420434349442066616907
:1075C0006C656400F0B591B000253EE000221146E4
:1075D00020A000F063FA322632E04121684600F034
:1075E00095FC0446002C27D06846FDF7C0FC0446F5
:1075F0001BA1684600F0E8FA00280ED1241F22469D
:1076000000A902311748FDF761FC102C02D20021BD
:1076100014480155012011B0F0BD112C10D1A41E49
:10762000224669460F48FDF751FC102C02D200217A
:107630000C4801550220EEE701200B4FBC4600DF4D
:107640003046761E0028C8D16D1C322DBEDB0020CE
:10765000E1E7000041542B47534E0D0A00000000A3
:1076600030780000B9080020C5B50008F0B589B031
:10767000002644E00022114623A000F00FFA322039
:10768000089034E01E21684600F040FC0546002DBD
:1076900029D06946002002F033FA1EA1684600F0A6
:1076A00093FA002823D1002414E0A01C6946085C4A
:1076B0000D2807D1102C02D20021174801557D2436
:1076C000E40006E0102C04D2A01C6946095C1248B4
:1076D0000155641C00A80230FDF749FCA042E4D823
:1076E000012009B0F0BD01200C4FBC4600DF089816
:1076F000411EC9B208910028C4D1701CC6B2322EF6
:10770000B8DB0020EDE7000041545E4D4549440DD3
:107710000A00000030780000A9080020C5B5000864
:10772000F0B5A1B000201E905AA102F0E9F90026A0
:1077300000201F90A7E0002E05D10022114659A07D
:1077400000F0ACF904E00022114658A000F0A6F9C0
:10775000322020908DE0412101A800F0D7FB0546A2
:10776000002D7CD0002E15D153A101A800F02CFAD9
:10777000002803D101A902F0C3F97AE052A101A8BF
:1077800000F022FA002874D101A902F0B9F9701CA6
:10779000C6B274E04EA101A800F016FA002803D189
:1077A00001A902F0ADF964E04EA101A800F00CFAC5
:1077B000002804D101A902F0A3F921B0F0BD4AA12B
:1077C00001A800F001FA002853D101A902F098F9AC
:1077D00000201290002440E001A8005D5F283BD10A
:1077E0001298401CC0B21290129801280AD101A927
:1077F000E01C095C10A8017301A9201D095C10A8F8
:10780000417329E01298032826D101A9A01C095C24
:1078100010A8817301A9E01C095C10A8C17301A91B
:10782000201D095C10A8017401A9601D095C10A845
:1078300041740021817413AB2FA21E2116A803F0FE
:10784000F9FA16A9002002F05BF913A8FDF7C0FBB6
:1078500007462D49FDF7B3FB641C01A800E004E0D6
:10786000FDF785FBA04204D9B6E70120274FBC46AF
:1078700000DF2098411E2091002800D06BE700BF58
:107880001F98401C1F901F980A2800DA53E700BF7A
:1078900093E700005B30335D4D6F64656D496E6644
:1078A0006F3A00004154490D0A00000041542B4C2E
:1078B000435453570D0A00004D616E756661637441
:1078C000757265723A0000004D6F64656C3A000095
:1078D000536F66747761726556657273696F6E3A3D
:1078E0000000000041503A00496E6E6572566572A4
:1078F00073696F6E3A0000005B30335D4D6F6465F5
:107900006D5665723A257300FE190020C5B5000852
:10791000F0B59FB000245CE03220149000221146A4
:1079200033A000F0BBF84CE0412102A800F0EEFAD1
:107930000646002E41D032A102A800F045F90028E9
:107940003FD102A8FDF713FB06B2002013900024DC
:1079500030E002A8005D0D281AD1002115AA139865
:10796000115415A8FDF734FB05B202A82B4627A237
:107970002821009015A803F05DFA15A9002002F057
:10798000BFF8A9B22648C172090A01731FB0F0BD41
:1079900002A8005D30280BDB02A8005D392807DC57
:1079A00002A8025D1398411C09B2139115A90A544B
:1079B000601C04B2B44204DACBE70120194FBC4684
:1079C00000DF1498411E09B214910028ACD1601C4C
:1079D00004B2052CA0DB2B4613A2282115A803F026
:1079E00029FA15A9002002F08BF800BFCEE70000AD
:1079F00041542B504F435F5645523F0D0A00000043
:107A00002B504F435F5645523A0000005B30345DC7
:107A1000504F437665723A25643C2D3E2573000035
:107A2000F8190020C5B500085B30345D506F63560F
:107A300065723D25640D0A00B0B500240AE00022FD
:107A4000114610A000F02AF83220124FBC4600DF89
:107A5000601CC4B2022CF2DBFF202D300D4FBC465F
:107A600000DF012040030C49088140100A492039F9
:107A700088610A20BC4600DF012000030649088116
:107A8000B0BD000041542B5A5057524F46460D0A84
:107A900000000000C5B5000820040048F8B50646FF
:107AA0000F461446002C08D13046FDF760FA85B227
:107AB0002946304602F088FB03E03946304602F0A2
:107AC00083FBF8BD70477047F0B593B0002639E0EE
:107AD0003220129000BF002211461EA0FFF7DEFFE9
:107AE00028E0412101A800F011FA0446002C1DD025
:107AF0001DA101A800F068F800281BD104A80130DE
:107B0000FDF766FA05461C498D4209D00022114650
:107B10001AA0FFF7C3FF01201F4FBC4600DFDAE7C2
:107B20001EA1002001F0ECFF13B0F0BD01201A4FA0
:107B3000BC4600DF1298411EC9B212910028D0D174
:107B4000701CC6B2052EC3DB19A1002001F0D8FFBE
:107B500000BFE9E741542B4C53485454535350450C
:107B600045443F0D0A0000002B4C534854545353D6
:107B7000504545443A000000581B000041542B4C2E
:107B8000534854545353504545443D2D312C3730C0
:107B900030300D0A00000000C5B500085B30365DCE
:107BA000536574545453205370656564204F6B00C3
:107BB0005B30365D5365745454532053706565646F
:107BC000204661696C65640030B502460B46194673
:107BD000144607E008782578A84201D0012030BD7E
:107BE000491C641C08780028F4D100BFF7E70000A6
:107BF00088B07848007840084000401C75490870FB
:107C0000012001F0C7FD74A1002001F079FF2020C0
:107C10007549886100F050F9002804D073A1002054
:107C200001F06EFF12E020206F492031088171A120
:107C3000002001F065FFFEF7E9F806E00020724938
:107C400008726420714FBC4600DFF7E701206E49DF
:107C50004871002211466EA0FFF720FF6EA10020A0
:107C600001F04EFFFFF75CFD5A48801DFDF79DF9BE
:107C700005462A466CA1684603F0F2F869460020E2
:107C800001F03EFFFFF744FEFFF79CFC00280AD0FE
:107C9000684B69A21E21684603F0CCF869460020B3
:107CA00001F02EFF03E068A1002001F029FFFFF79B
:107CB0000BFF4CA1002001F023FF02F069FF49A156
:107CC000002001F01DFF01F0D1FE64A1002001F0B1
:107CD00017FFFFF7B9FB43A1002001F011FFFFF7E9
:107CE000A1FA40A1002001F00BFFFFF703FA3DA12C
:107CF000002001F005FF01F0E5FD3AA1002001F0B0
:107D0000FFFE202038492031088161E0C821594810
:107D100000F0FCF804462F480078C007C00F002888
:107D200007D1002C04D10120384FBC4600DF4FE0C2
:107D30004EE0002C14D04F4800782B2803D04D483B
:107D400000785E280BD100202F490872494901F0C4
:107D5000D7FE484800F034FE4648FDF71BFC37E0EC
:107D600001202A4FBC4600DF27480078002803D1B5
:107D7000012001F00FFD16E023488078002803DD84
:107D8000032001F007FD0EE01F480079002807DD01
:107D90001D488079002803DD042001F0FBFC02E08F
:107DA000022001F0F7FC02F0C9FF334800683349B4
:107DB0000968884200D20BE02F480068FF302D3060
:107DC0002E490860002211462DA0FFF767FE00BF74
:107DD0009CE70000F81900204D6F64656D496E69DD
:107DE000742E2E2E0D0A000000040048204F4B0D6B
:107DF0000A000000204661696C0D0A47545F4D6F10
:107E000064650D0A00000000BC110020C5B5000823
:107E1000415445300D0A00005B30325D415445301D
:107E2000204F4B0D0A0000004D5F5665723A2564E5
:107E30000D0A0000B90800205B30355D494D454909
:107E40003A25730D0A0000005B30355D494D454908
:107E50003A4661696C65640D0A0000005B385D5349
:107E6000696D43617264436865636B206F4B0D0AF3
:107E700000000000091A002078010020680100209D
:107E800041542B434353510D0A0000000021064882
:107E9000064FBC4600DF06E005490348054FBC46D7
:107EA00000DF02F049FBF7E76001002067B9000836
:107EB000FFFF0000E5B9000880B500F0FBF80120E5
:107EC00000031049886164200F4FBC4600DF012089
:107ED00000030C492031088140000A498861642070
:107EE000BC4600DF0120400306492031088102F032
:107EF000E1FD02F0C7FE002801D0002080BDFFF7A1
:107F0000B5FBFBE700040048C5B50008F8B5074617
:107F10000B462C498888002800D1F8BD488880008D
:107F20008E1D365A68460680488880008E1D80194E
:107F30004688684646800024002223E05820405AA4
:107F4000002800D122E05C26765A086E855D5C2010
:107F5000405A401C5C2670525C20405A5626765A85
:107F6000B04202DB00205C2670525820405A401E6E
:107F7000582670529C4203DA2046661CB4B23D5427
:107F8000501C82B2684600889042D7DC00BF488807
:107F9000401C48804888142801DB002048808888DD
:107FA000401E888068460088904201D0FE20B4E7D9
:107FB00068460088984201DDFF20AEE768460088E9
:107FC000C0B2AAE75811002070B503460A4612480D
:107FD0000024048084804480002108E000258E0075
:107FE000841D341965808E00841DA553491C1429F5
:107FF000F4DB0366002103E00024056E6C54491C89
:108000009142F9DB5624225200255A2425525C2441
:1080100025525824255270BD5811002070B50446D1
:108020000A4623498888142801DBFF2070BD5820A8
:10803000405A85185620405A854201DDFE20F5E75A
:108040005A20455A08888600881D301845800888BF
:108050008500881D425300231AE0E55C5A20405AEF
:108060000E6E35545A20405A401C85B25A20455253
:10807000405A5F25ED00A84202DB00255A204552F8
:108080005820405A401C85B258204552581C83B293
:108090009342E2DB0888401C08800888142801DB32
:1080A000002008808888401C88800020BEE70000EF
:1080B0005811002000B55F21C9000248FFF784FF76
:1080C00000BD0000600E0020704700000021827893
:1080D000002A27D0184A03231B02D21803789B10CA
:1080E0009B00D15802789207D30EFF229A400B468C
:1080F0009343194642789207120E03789B07DB0ED2
:108100009A4011430C4A03231B02D21803789B1098
:108110009B00D1500278D306DB0E01229A40064B19
:108120001A6007E00278D306DB0E01229A40024B68
:1081300080331A607047000000E100E010B50028AD
:1081400019DA1A4A03071B0F083B9B089B00D258F9
:108150008307DC0EFF23A3409A438B071B0E840783
:10816000E40EA3401A43114B0407240F083CA40853
:10817000A4001A5118E00E4A03231B02D2188308E8
:108180009B00D2588307DC0EFF23A3409A438B0742
:108190001B0E8407E40EA3401A43054B032424025C
:1081A0001B198408A4001A5110BD00001CED00E04A
:1081B00000E100E0F3B583B00C460398FCF7D7FE6E
:1081C00007463A461AA1684602F04AFE6946002070
:1081D00001F096FC0025002622E0332228466D1C83
:1081E00022540398825D28466D1C22543022284672
:1081F0006D1C225428466D1C2254781EB04200D1BA
:1082000010E0322228466D1C2254302228466D1C74
:10821000225428466D1C225428466D1C2254761C7C
:10822000BE42DADB00BF0020605505B0F0BD0000A3
:108230006C656E3D25640D0A00000000704700006B
:1082400010B5024600200D4B1868800880000346D8
:1082500013431846094B1860094B1B690424234338
:10826000074C2361012901D130BF00E020BF044B3E
:108270001B690424A343024C236110BD007000401D
:1082800000ED00E0002905D0054A52680243044B86
:108290005A6004E0024A52688243014B5A607047B8
:1082A00000700040F0B5F7B005463822FD4969A8D6
:1082B000FCF70CFE0020039000BF0398411C8000D7
:1082C000039169A9085800780028F6D10398401E48
:1082D0000390002625E0B00069A908580590E81C25
:1082E000049000200690079011E00598017804980A
:1082F0000078814202D0012006900CE00598401CD5
:1083000005900498401C04900798401C079005981D
:1083100000780028E9D100BF0698002800D103E0CA
:10832000761C03988642D6DB00BF0398864201D1B3
:1083300077B0F0BD330002F0A7FD0D0813143567C8
:10834000D1F0EFEEEDECEBEA1200092001F052FA69
:10835000D5A1002001F0D4FB0220FDF7B3F9BFE264
:10836000BEE2092001F046FAD2A1002001F0C8FBCC
:108370000220FDF7A7F91020D14908814020D049FB
:1083800020398861FFF79EFBFFF79DFB012040032A
:10839000CB492039886140108861C9490881FDF7BF
:1083A000B3FE9DE2092001F025FA287A4D2810D16C
:1083B000687A43280DD1A87A55280AD1C1A1002096
:1083C00001F09EFB5520C349487001F09FF900BFA2
:1083D000FEE7287A4D2816D1687A4F2813D1A87A5B
:1083E000442810D1E87A45280DD1287B4D280AD1A0
:1083F000B9A1002001F084FB00221146BAA0FFF7CA
:108400004DFBFDF781FE6BE24EAABCA12846FDF7AD
:108410008BFF0446012C01DB282C00DB60E24EA917
:1084200012A8FCF7B9FD4EAAB5A12846FDF77CFFBE
:108430000446002C01D1689007E0052C00DD4FE2D6
:108440004EA8FCF7C5FD80B268904EAAAEA12846A2
:10845000FDF76AFF0446012C01DB142C00DB3FE230
:108460004EA90DA8FCF798FD4EAAA9A12846FDF734
:108470005BFF0446012C01DB142C00DB30E24EA92B
:1084800008A8FCF789FD08A80DAB12AAA3A10090CB
:108490004EA802F0E5FC00221CA94EA8FDF738F812
:1084A00000221146A2A0FFF7F9FA002211461CA8EB
:1084B000FFF7F4FA002211467DA0FFF7EFFA08A8B3
:1084C0000DA90091019012AA9DA14EA8689B02F0EF
:1084D000C7FC4EA9002001F013FB01E24EAA87A1C0
:1084E0002846FDF721FF0446012C01DB282C00DB88
:1084F000F6E14EA912A8FCF74FFD4EAA80A128462E
:10850000FDF712FF0446002C08D168900EE0DBE175
:108510009CE1B6E0A4E081E06CE06AE0052C00DDBF
:10852000DEE14EA8FCF754FD80B268904EAA90A1FF
:108530002846FDF7F9FE0446012C01DB0A2C00DD7C
:10854000CEE14EA8FCF751FD679062491D31679856
:10855000FCF735FD12A95F482130FCF71DFD5D4990
:108560006898C875000A087608467130FCF7FFFC69
:108570000E2804D27FA1002001F0C2FAB0E15548D4
:108580001D30FCF712FD0746524871303B4612AAD7
:108590007FA100904EA802F063FC00221CA94EA807
:1085A000FCF7B6FF002211467FA0FFF777FA002202
:1085B00011461CA8FFF772FA002211463CA0FFF7F3
:1085C0006DFA01F0A3F843481D30FCF7EEFC009073
:1085D0004048017EC27D0802104303463D4A2132D5
:1085E00075A14EA802F03CFC4EA9002001F088FACB
:1085F00076E175E137481D30FCF7D7FC0746354872
:108600002130034650333A4673A100904EA802F041
:1086100027FC4EA9002001F073FA61E1092001F066
:10862000E9F87DA1002001F06BFA01207D4FBC46E6
:1086300000DF0220FDF746F8FFF744FA012040036F
:108640001F49088140101E49203988610520BC4619
:1086500000DF012000031A490881FDF755FD3FE1C5
:108660001C48817D427D080210430346194AD21DF1
:108670006DA14EA802F0F4FB4EA9002001F040FAD3
:108680002EE16D48837841781806001408430246AD
:108690006AA14EA802F0E4FB4EA9002001F030FAD6
:1086A0001EE10000CCBD000847542B544D3A4F4BFF
:1086B0000D0A000047542B444D3A4F4B0D0A000061
:1086C0002004004847542B464F54413A4D43550D22
:1086D0000A0000003808002047542B464F54413A06
:1086E0004D4F44454D0D0A0061742B706F633D3151
:1086F000303030303031380D0A0000004950000071
:10870000506F7274000000004163636F756E7400F7
:1087100050617373776F72640000000069703D25CB
:10872000733B69643D25733B7077643D25733B0063
:1087300041542B504F433D31323030303000000037
:1087400047542B5354503A49503D25733B506F7258
:10875000743D25753B4163636F756E743D25733BB6
:1087600050617373776F72643D25730D0A000000CA
:1087700050534E0047542B534D503A4641494C5BA1
:108780004D45494420496E76616C69645D0D0A006F
:1087900069703D25733B69643D256C753B7077645A
:1087A0003D25733B0000000041542B504F433D30AA
:1087B000313030303000000047542B534D503A498F
:1087C000503D25733B506F72743D25753B50534EA1
:1087D0003D256C750D0A000047542B524D503A5000
:1087E000534E3D256C753B4D4549443D25733B43F8
:1087F0004E554D3D303030303030303030303B55DC
:10880000494D49443D303030303030303030303BED
:1088100049503D25730D0A0047542B5053543A4F8D
:108820004B0D0A00C5B5000847542B5645523A2552
:10883000735F5625640D0A00E812002047542B424E
:1088400041543A20256420560D0A00004EAA2649BC
:108850002846FDF769FD0446012C01DB0F2C00DDE5
:1088600066E54EA90DA8FCF797FB4EAA1E490831F4
:108870002846FDF759FD0446012C01DB0F2C00DDD5
:1088800056E50DA91948FCF787FB4EA9174810308B
:10889000FCF782FB00F03AFF144B1033134A14A18B
:1088A0001CA802F0DDFA1CA9002001F029F90F4BE9
:1088B00010330E4A17A11CA802F0D2FA012200219F
:1088C0001CA8FFF7EBF80BE0084B1033074A16A182
:1088D0001CA802F0C5FA1CA9002001F011F900BF84
:1088E00000BF00BF24E5000008870008D908002069
:1088F00047542B41504E3A4163636F756E743D256A
:10890000733B50617373776F72643D25733B0D0A3F
:108910000000000041542B5A5049445057443D2513
:10892000732C25730D0A000047542B5241504E3AC8
:108930004163636F756E743D25733B50617373774C
:108940006F72643D25733B0D0A000000F0B58FB0D7
:1089500006460020019000250027019014E0745D78
:10896000302C01DB332C00DD13E06D1C745D302CEA
:1089700001DB332C00DD0CE0332C01D1781C87B2F5
:108980006D1C0198401C0190FF212D3101988842F7
:10899000E5DB00BF064847813A4606A102A802F07F
:1089A0005FFA02A9012001F0ABF80FB0F0BD0000A2
:1089B000BC1100205B4F4C557365723D25645D0012
:1089C00070B59EB0044660784C2818D1A078532822
:1089D00015D1E078482812D1207954280FD1607A37
:1089E00045280CD10020F749C87008468078002837
:1089F00002D10120F449886101201EB070BD607968
:108A0000302829D1A079422826D1E07946280FD1F3
:108A1000207A46280CD10020EC4908700120EA4950
:108A2000203108810C219320C00000F083FE11E06A
:108A3000E07930280ED1207A30280BD10120E1498D
:108A40000871E2490870E049203108810C21E048B2
:108A500000F070FE0120D0E76079382870D1A0794D
:108A600042286DD1E07930286AD1207A31280ED1A0
:108A70000120D44908710220D64908810020D1493B
:108A800088700120D0498861CE49087009E0207AB9
:108A9000302806D10020CB49087102200921C906DF
:108AA0008861607A30281ED1A07A30281BD1C7484F
:108AB000007801280BD10020C4490870C148807893
:108AC000002802D00020BF498870012095E70020CF
:108AD000BC4988700120BC49203108810C21BC4868
:108AE00000F028FE29E0607A30280ED1A07A3128E3
:108AF0000BD10120B34908708870B3492031088137
:108B00000C21B34800F016FE17E0607A312814D12A
:108B1000A07A332811D1AD480078012802D1002075
:108B2000AA4908700120A7498870A7492031088107
:108B30000C219320C00000F0FDFD01205DE7FFE760
:108B40006079382878D1A0793228FBD1E17968465C
:108B50000170217A417000218170FCF739FAC6B2A8
:108B6000002E06D0012E73D0022E76D0032E6ED1A9
:108B700099E000209349087097A1684602F070F9C7
:108B8000607C422829D1A07C352826D1607E4328EC
:108B900023D1A07E412820D18A484078002808D1DE
:108BA00000228FA10120FEF771FA01219348417242
:108BB0000EE09248C0793C280ADB00218F48C17141
:108BC000002287A10120FEF761FA01218B48417242
:108BD0008BA16846FCF79EF935E0607C43282ED1D6
:108BE000A07C45282BD1607E432828D1A07E322846
:108BF00025D174484078002809D18048407A00285F
:108C000015D1002282A10120FEF740FA0FE07B4837
:108C1000007A3C280BDB7948407A002807D10021F4
:108C20007648017200227AA10120FEF72FFA7EA178
:108C30006846FCF76FF906E03DE009E00DE07DA134
:108C40006846FCF767F96946002000F059FF2FE0FD
:108C50007BA1002000F054FF2AE020461130FCF7F1
:108C600086F9801EC5B2512D00DB51252A462146CA
:108C7000113154482030FCF76DF9512D03DA0021F1
:108C8000504820304155002060740922A1184D48F9
:108C90000E30FCF75FF96DA1002000F031FF0120DC
:108CA0006D49087004E06DA1002000F029FF00BFAD
:108CB00000BF0120A1E6607938285CD1A079362870
:108CC00059D101203F490870207A30284FD12046E1
:108CD0001130FCF74CF9801EC5B2512D00DB512537
:108CE0002A462146113137487130FCF733F9512DAE
:108CF00003DA0021334871304155002060740922A5
:108D0000A11830481730FCF725F92E484078002884
:108D10001BD151480078002806D12A4A713252A14D
:108D2000684602F09DF80AE000204B490870254B88
:108D300071331A46513A4DA1684602F091F801226A
:108D400069461046FEF7A2F911E04E480078012866
:108D50000DD100204B4908701A4A71324AA1684669
:108D600002F07EF8002269460120FEF78FF901200B
:108D70001449487041E6607938280AD1A07933282F
:108D800007D1E079302804D1207A302801D10120A0
:108D900033E6607938280AD1A079332807D1E07901
:108DA000302804D1207A312801D1012025E66079CC
:108DB000392872D1A07931286FD1E01DFFF7C6FDA7
:108DC00001201AE6BC110020000400483F010020E9
:108DD0006E030000200000485B6D73675D000000BB
:108DE00044354341424143354430433543464132A3
:108DF000423445444345463300000000DC12002065
:108E00004C6F67696E206661696C656400000000E4
:108E10004345444543444638433245374331414353
:108E200042444433000000004E6F206E6574776F3B
:108E3000726B00004E6F206C6F67696E000000005F
:108E40006C6F67696E20696E670000006C6F676900
:108E50006E206F6B000000003E0100206C6F676F9A
:108E6000757420696E670000257300002573324316
:108E7000443244314235433743324244324325730E
:108E8000000000003D01002042444638433845427E
:108E90003243257300000000FFE76079302804D1D9
:108EA000A079652801D10120A7E5607938280DD186
:108EB000A07934280AD12046FEF7D4F801222146B1
:108EC00009311046FEF7E2F8012096E56079322874
:108ED00015D1A079312812D12046FEF7C3F801221E
:108EE000214615311046FEF7D1F8002060750922A1
:108EF00021460D311448FCF72DF801207DE56079FD
:108F000031281FD1E07930281CD1A07B372802D02E
:108F1000A07B382816D109210B480930FBF7EFFF59
:108F200009222146133108480930FBF7CFFF2046BC
:108F3000FEF798F8002221461F310120FEF7A6F81F
:108F400001205AE5002058E5CF12002070470000AC
:108F50000C4949680122920391430A4A5160114623
:108F6000496882B21143074A51601146096B921554
:108F70009143044A11631146096B020C1143014AE3
:108F80001163704700100240002905D0054A52695C
:108F90000243044B5A6104E0024A52698243014B86
:108FA0005A61704700100240002905D0054AD26975
:108FB0000243044BDA6104E0024AD2698243014B66
:108FC000DA61704700100240002905D0054A926915
:108FD0000243044B9A6104E0024A92698243014BC6
:108FE0009A61704700100240002905D0054AD268F6
:108FF0000243044BDA6004E0024AD2688243014B28
:10900000DA607047001002400348406A01210906F7
:1090100008430149486270470010024010B50446F9
:1090200021462F204004FFF7AFFF10BDFEB50446D8
:10903000002500260020019000900027504840683D
:109040000C2108400546002D04D0042D05D0082D24
:1090500028D105E04B48206027E04A48206024E002
:10906000474840680F218904084006464448406844
:109070000121090408400190B00C861C01980028C9
:1090800003D14148704320600BE03D48C06A0007AF
:10909000000F401C00903B480099FBF7EDFE704329
:1090A000206002E03748206000BF00BF34484068BD
:1090B000F021084005462D093448475D2068F840F6
:1090C00060602F48406807210902084005462D0AC4
:1090D0002E48475D6068F840A0602948006BFF217A
:1090E00001310840884202D02948E0600DE0244860
:1090F0004068012189030840884203D0A0684008E5
:10910000E06002E0A0688008E0601D48006B40213C
:109110000840402802D01F48206102E00120C0031F
:1091200020611748006B10210840102802D0154814
:10913000606101E0206860611148006B8007800F6A
:10914000002802D1A068A06119E00D48006B8007DB
:10915000800F012802D12068A06110E00848006B50
:109160008007800F022802D18003A06107E0044835
:10917000006B8007800F032801D10248A061FEBD6B
:109180000010024000127A0000093D00E8000020B3
:10919000809FD5001280000010B5024600210023F8
:1091A00000205111002902D10C4C23680BE0012949
:1091B00002D10A4C236A06E0022902D1074C636AF5
:1091C00001E0064C636BD106C90E01248C401C40A3
:1091D000002C01D0012000E0002010BD0010024052
:1091E0007047F7B505460B46002600240BE028190A
:1091F00000F05AFA02463046761C1A5410123146D4
:10920000761C5854A41C02988442F0D3FEBD000082
:1092100070B500240025C8223D493E48FFF7E1FF14
:109220003B48007848280AD139484079A84206D1FD
:1092300039A13748C01DFBF7A1FE002848D038A14E
:10924000002000F05DFCC8213148FBF758FE4820A3
:109250002F490870882048700020887048718871F4
:109260002DA12B48C01DFBF797FE6F2128484175A3
:10927000002181752D49C175090A01762B49C91C48
:10928000C176090A017701461D312948FBF797FE8F
:1092900028A11F482130FBF77FFE2AA11C4871300E
:1092A000FBF77AFE2BA11A489130FBF775FE2BA134
:1092B0001748A130FBF770FE28A11548B130FBF725
:1092C0006BFE00211248C1300171417101240FE091
:1092D0000F48817D427D080210436F2808D06F211E
:1092E0000B48417500218175C13001714171012424
:1092F000002C01D000F00AFA05491D311948FBF78E
:109300005EFE19A102482130FBF746FE70BD000049
:109310003808002000FC00084B4644333138000078
:1093200052737420506172610D0A00006E050000D6
:10933000BB11A6763132312E3230352E322E3638F0
:1093400000000000303030303030303030303030DD
:109350003030000063746E657400000063617264F5
:1093600000000000A81877093138332E3133312E30
:1093700031332E313000000010B598B03548FBF77E
:1093800014FE3549884205D33248FBF70EFE401CD7
:10939000002806D1012231A10320FDF777FE18B085
:1093A00010BD2C48FBF701FE04462A4A54322146E0
:1093B00015A8FCF7B3FE00281CD015AA2EA101A801
:1093C00001F04EFD01A9002000F09AFB01A915A8AB
:1093D000FEF7F0FE002211462BA0FEF75FFB0022F5
:1093E000114601A8FEF75AFB002211462DA0FEF7F8
:1093F00055FB08E02CA1002000F082FB0022114662
:109400002DA0FEF74BFB1348FBF7CFFD0446224689
:1094100034A115A801F024FD15AA33A101A801F07B
:109420001FFD01A9002000F06BFB01A915A8FEF7A4
:10943000C1FE002211462FA0FEF730FB002211468C
:1094400001A8FEF72BFB002211462FA0FEF726FBFA
:1094500000BFA4E7550800202058F20843383745DC
:109460004546374131363746463735333139393558
:109470004546384200000000436865636B436F64F3
:10948000653D25730D0A000041542B4C534854543C
:10949000533D312C22443041334431453943324528
:1094A0004200000032430000436865636B436F6411
:1094B000653D4E554C4C000041542B4C5348545480
:1094C000533D312C224430413344314539433245F8
:1094D00042424246314338413143414137423044B0
:1094E00043324300256C750050534E3D25730D0AE1
:1094F0000000000044364435423643424231453094
:109500004332454200000000220D0A0000B593B02E
:10951000064B1A46513A06A101A801F0A1FC01220E
:1095200001A91046FDF7B2FD13B000BD2D120020B9
:10953000257332432573000010B5AAB00F498B780C
:109540004A78190609141143084609A9FCF79CFF3B
:109550000B48FBF72AFD044601A9FCF7CBFF01A845
:1095600009AB08A26421009011A801F063FC01225C
:1095700011A90320FDF78AFD2AB010BDE8120020D2
:10958000051A0020333537354346393137453736EC
:1095900030363532344234452573257300000000DF
:1095A00010B5AAB02AA111A801F05AFC2D48817D5E
:1095B000437D0802184302462BA102A801F050FC8B
:1095C000002207A902A8FBF7A3FF07A911A8FBF730
:1095D000A1FC26A111A8FBF79DFC2A48FBF7E5FC9E
:1095E00004462848801F017BC27A080210430346C4
:1095F000224625A102A801F033FC002207A902A8F7
:10960000FBF786FF07A911A8FBF784FC012211A92B
:109610001046FDF73BFD1B48FBF7C7FC0446194805
:10962000801F017BC27A0802104300900D48817DA3
:10963000437D080218430246234615A111A801F0F4
:109640000FFC11A9002000F05BFA2AB010BD000049
:109650004433413644334333423045364231424548
:1096600032430000380800202564000032434334B0
:109670004133424645394230453642314245324314
:1096800000000000FE19002025642C256400000065
:10969000415665723D25642C4D5665723D25642CFE
:1096A000505665723D2564000146088870470000E9
:1096B00030B500228B071C0F0F23A3401A460B4B1B
:1096C0008C10A4001B599343084C8D10AD006351BE
:1096D00023468C10A4001B598C07250F0446AC4070
:1096E0002343024C8D10AD00635130BD0800014092
:1096F00001460020044A10688008800002460A43A0
:109700001046014A106070470000014010B520204B
:1097100005498861C8220549054801F045FB20201C
:1097200001492031088110BD00040048380800209C
:1097300000FC000870B505460C4601200A49088166
:109740002146284600F06CFB0120084908700021E2
:1097500006484170817006480088201881B203488D
:10976000C170090A017170BD200400482501002064
:109770007801002043185A00FF2A00DD7047034B90
:109780001870034B197000BFF8E70000FA000020C2
:10979000FB00002010B50446230001F075FB050412
:1097A0000B1219202700002011490870012000F039
:1097B00021F81BE001200E490870052000F01AF87E
:1097C00014E002200A490870062000F013F80DE0AA
:1097D000032007490870042000F00CF806E004207C
:1097E00003490870012000F005F800BF00BF10BD5C
:1097F000FC00002010B50446230001F045FB0A06DA
:109800000F18212A333C454E57600021084600F0CE
:10981000B1F800210846FFF7ADFF50E0002101201C
:1098200000F0A8F800210846FFF7A4FF47E0012157
:10983000084600F09FF800210846FFF79BFF3EE036
:109840000A21012000F096F800210846FFF792FF58
:1098500035E00021084600F08DF800210120FFF7D7
:1098600089FF2CE00021084600F084F80121084619
:10987000FFF780FF23E00021084600F07BF80A2173
:109880000120FFF777FF1AE00021012000F072F8B5
:1098900000210120FFF76EFF11E00121084600F0D2
:1098A00069F801210846FFF765FF08E00A21012059
:1098B00000F060F80A210120FFF75CFF00BF00BF45
:1098C00010BD0000F0B591B0002523E03226002243
:1098D000114614A0FEF7E2F815E041216846FEF7B4
:1098E00015FB0446002C0AD013A16846FEF76CF95C
:1098F000002808D114A100F003F911B0F0BD012037
:10990000164FBC4600DF3046711E0EB20028E4D16F
:10991000681C05B2052DD9DB11A1002000F0F0F87C
:1099200000BFEAE741542B504F433D3130303030D7
:109930003032300D0A0000002B504F433A313030A6
:1099400030303030300000005B31345D53696D7071
:109950006C654D6F64655F4F6B000000C5B5000816
:109960005B31345D53696D706C654D6F64655F5438
:109970006F75740043185A00FF2A00DD7047034BCF
:109980001870034B197000BFF8E70000F8000020C2
:10999000F90000200CB500200190009031480068CB
:1099A0000121090408432F49086000BF2D480068C1
:1099B00001214904084000900198401C0190009842
:1099C000002804D10521090201988842EED12548DA
:1099D0000068012149040840002802D001200090BD
:1099E00001E0002000900098012839D111201E4983
:1099F00008601C4840681B49486008464068486049
:109A0000084640683F2109048843164948600846D3
:109A10004068052109040843124948600846006867
:109A20000121090608430F49086000BF0D4800687E
:109A30000121490608400028F8D00A4840688008FB
:109A400080000849486008464068022108430549EB
:109A5000486000BF034840680C2108400828F9D13D
:109A60000CBD0000001002400020024090B58DB0F7
:109A7000184CFDF77BFC00282AD128E032216846EB
:109A8000FEF744FA002800D021E00120124FBC4626
:109A900000DF00201149087211480078C007C00F8C
:109AA000002800D113E0601C80B204467D2109012A
:109AB000884201DB002400E009E00AA1002000F058
:109AC0001FF801220AA10320FDF7E0FA00BFD5E745
:109AD0000DB090BDDC050000C5B50008BC1100202C
:109AE000F81900204E6F20636172640D0A000000B7
:109AF00046373842443236333631353300000000C1
:109B000070B506460D4609480078002800D070BDA3
:109B10002846FBF72CFA84B2C82C00DDC824214665
:109B2000284600F0F7FA00BFF1E700002C01002002
:109B300030B502460B461946144607E008782578EA
:109B4000A84201D0012030BD491C641C08780028BF
:109B5000F4D100BFF7E7000010B50120FFF75EFA6F
:109B600064211D480068FBF787F904461B488442BE
:109B700000D90EE02002000A401E19494861032165
:109B8000081FFEF7DBFA00201549886107200861ED
:109B900000BFFBF72DFCFCF77DFEFDF70DF8FDF790
:109BA00047FCFFF7D3F9FEF749FBFBF7F9FCFBF79E
:109BB000C3FF00F017FFFDF75BF9FBF763FB00BF86
:109BC000FCF7FCFB07494870020A8A700028F7DBA3
:109BD0000120FCF7EDFC10BDC4000020FFFFFF00DA
:109BE00000E000E0E812002010B521480078C0072E
:109BF000C00F002819D01E480179C278080210430E
:109C00001C490968884210D800211B4800F09EF8C2
:109C100000201749087019488078002805D118A13C
:109C2000FFF76EFF01201849886118480078400747
:109C3000C00F00281BD01548801CFBF7B6F90D4952
:109C40000968884213D211480078042188430F49DB
:109C500008700A488078002809D10848C078002890
:109C600005D10BA1FFF74CFF01200749886110BD0A
:109C7000250100207801002000480140BC1100208F
:109C800054455354310D0A0000040048F8190020CF
:109C900054455354320D0A0010B520200A4908815A
:109CA00000210A48FBF7BEFAFCF79CF901210807DE
:109CB000FFF77AF901210802FEF7E4FA01210846CC
:109CC000FEF7BEFA10BD0000200400480024014049
:109CD00010B51B480068012108431949086008466F
:109CE0004068184908401649486008460068164907
:109CF0000840134908600846006801218904884328
:109D00000F490860084640683F21090488430C4910
:109D100048600846C06A00090001C8620846006B36
:109D2000FF2154318843064908630846406B4008C8
:109D30004000486300208860FFF72CFE10BD000043
:109D4000001002400CB8FFF8FFFFF6FE002904D017
:109D5000028801231A43028003E00288014B1A4063
:109D600002807047FEFF0000002907D04422125AEB
:109D70000123DB031A4344231A5205E04422125AFA
:109D800053045B0C442213527047000070B500244A
:109D900000220023058C1C4E35400584028C8388EC
:109DA000048B194D6F3D2C40B51E2C400D882C4363
:109DB000751E2A408D892A434D882A43134DA84297
:109DC00008D0134DA84205D0124DA84202D0124D22
:109DD000A84212D10C4DED1F2A40CD892A430A4DCD
:109DE000ED1E2A408D882A43074DFF3D2B400B4D29
:109DF0002B400D8A2B434D8A2B43838004838D682F
:109E00004563028470BD0000FEFF0000002C01408D
:109E1000004001400044014000480140FFFD0000B7
:109E2000F0B589B005460F46002629461C48006853
:109E3000FBF722F8401E84B22046E10F09184E10AD
:109E400001218804FFF7C0F800216846018341839F
:109E50000794018408A8817006A9124800F024F82C
:109E60007021684681800121C18004210181022185
:109E7000018200214182FF21013181820021C182C2
:109E8000039601A90748FFF781FF01210548FFF765
:109E90005DFF01210348FFF767FF09B0F0BD000037
:109EA000C40000200048014000220288154B98425F
:109EB00006D001239B07984202D0134B984203D14E
:109EC000124B1A404B881A43114B984203D0114B46
:109ED0001A400B891A4302804B68C3620B880385C2
:109EE000084B984208D00C4B984205D00B4B984237
:109EF00002D00B4B984201D18B7A038601238382D7
:109F000070470000002C0140000400408FFF00005B
:109F100000100040FFFC00000040014000440140F0
:109F2000004801406A210848FAF7E9FF0021074884
:109F3000074FBC4600DF06E006490448064FBC4612
:109F400000DFFCF737FFF7E7B0070020E000002054
:109F500067B90008FFFF0000E5B9000838B52D4CCF
:109F60002D492E4800F0AFF9002813D02B4800F0FF
:109F70006DFAC0B200902849284800F07BF92848C3
:109F80000078022805D168460178264800F063FA77
:109F900000E000BF2449214800F095F900282BD0AB
:109FA00021491E4800F066F92048406BC8210D1A6F
:109FB00000211E483030FBF73BFC052D0FD92078DF
:109FC00047280CD16078542809D1A0782B2806D1D5
:109FD000A9B21048001F4170090A81700CE00021ED
:109FE0000C48001F41708170C8201049486301214E
:109FF0000E483030FBF71CFC0821084800F059F9E6
:10A00000012806D1054800F021FA0821034800F094
:10A010002FF938BD04090020050105000038014072
:10A020002C01002000440040040104000000024014
:10A0300008B53049304800F046F900284AD02E488B
:10A0400000F004FAC0B200902C480078022809D130
:10A05000684601782A4800F0FEF92649264800F0B3
:10A0600009F908BD27480179C278080210435F2129
:10A07000C900884227DA6846027822488179437904
:10A08000080218431F4909310A541E488179427950
:10A0900008021043401C81B21A4841710A0A8271B9
:10A0A0005F20C000814203DB0021164841718171AD
:10A0B00014480179C27808021043401C81B211484B
:10A0C000C170090A0171104801F076F909490A487E
:10A0D00000F0D0F80821084800F0EBF8012806D17C
:10A0E000054800F0B3F90821034800F0C1F800BFAB
:10A0F000B7E7000005010500004400402C010020E6
:10A1000000380140940A00206001002010B5FFF7DC
:10A1100025FF10BDF3B581B00D460024002D00D100
:10A12000FEBD04E01748C078002800D105E0601C9F
:10A1300080B2044614498842F4DB00BFC82D01DD1B
:10A14000C82600E02E460F4FCC37002404E00198CB
:10A15000005D3855601C84B2B442F8DB00210B4826
:10A16000FBF766FB0748CC3008491C398862084673
:10A17000066201200349C87001210448FBF758FB1F
:10A1800000BFCDE700090020E02E00001C000240C7
:10A1900010B52020FBF7AAFB01280CD11020FBF7FB
:10A1A00041FB2020FBF738FB00210348FBF740FB75
:10A1B00000200249C87010BD1C00024000090020A8
:10A1C00010B5FFF735FF10BD70B506460C46002CE4
:10A1D00001D0C82C00DD70BD04E014488078002850
:10A1E00000D105E0681C80B2054611498842F4DBC5
:10A1F00000BF002504E0705D0E494855681C85B21B
:10A20000A542F8DB00210C48FBF712FB09480A497C
:10A21000091F0861084684600120044988700121F3
:10A220000548FBF705FB00BFD5E70000940A0020B6
:10A2300060EA0000950D00204400024010B50120A6
:10A240004003FBF753FB01280DD10003FBF7EAFAAB
:10A2500001204003FBF7E0FA00210348FBF7E8FA8E
:10A2600000200249887010BD44000240940A00207A
:10A270000162704710B5002300220B0C01249C40A2
:10A280002246026210BD002904D0026801231A434D
:10A29000026003E002685208520002607047002A20
:10A2A00003D083680B43836002E083688B43836041
:10A2B000704702460020D3690B40002B01D00120DB
:10A2C00000E00020704770B502460B4600240021D4
:10A2D000002500201E04350ED9B201268E403146DD
:10A2E000012D02D11668314006E0022D02D15668D8
:10A2F000314001E0966831401C0C0126A6403446EE
:10A30000D6693440002903D0002C01D0012000E0A0
:10A31000002070BDF8B503460024002600960025F5
:10A32000002018460E04340ECEB200960127009E7F
:10A33000B7403D46022C01D1001D02E0032C00D1A4
:10A340000830002A03D006682E43066002E0066843
:10A35000AE430660F8BD0000F0B589B005460E4674
:10A3600000240020089000BF00BF2868400840007B
:10A3700028606C6803210903204688430446B068BE
:10A3800004436C602C682F480440F16870680843EF
:10A390003169084304432C60AC680321090220465C
:10A3A0008843044670690443AC606846FEF73EFE8D
:10A3B0002548854202D10698089001E0029808904D
:10A3C00028680121C9030840002809D032685100DB
:10A3D0001923089A5A431046FAF74EFD074608E03B
:10A3E000326891001923089A5A431046FAF744FD3F
:10A3F000074664213846FAF73FFD0401200964212D
:10A400004843381A079028680121C90308400028EA
:10A410000AD00799C900084632306421FAF72CFDAA
:10A420004007400F044309E007990901084632300C
:10A430006421FAF721FD0007000F0443AC8109B045
:10A44000F0BD0000F3E9FFFF003801400146888CB1
:10A45000C005C00D7047CA05D20D028570470000C7
:10A4600010B586B0044625480078A04202D02348A3
:10A47000047001E006B010BD002C20D0E1204002A5
:10A480000090002001900290039005900C20049011
:10A4900069461B48FFF760FF01211948FFF7F3FEEB
:10A4A000012218491648FFF735FF012240211448C0
:10A4B000FFF7F5FE01211448FBF7BAF91BE0E12094
:10A4C0004002009000200190029003900590082027
:10A4D000049069460A48FFF73FFF01210848FFF74B
:10A4E000D2FE002207490648FFF714FF0022402150
:10A4F0000348FFF7D4FE00BFBCE700003401002092
:10A5000000380140040104003000024070B50546E7
:10A510000E4600240BE0295D0648FFF79CFF00BFB4
:10A5200040210448FFF7C5FE0028F9D0641CB4425E
:10A53000F1DB70BD00380140F0B5FFB0C6B0C548D2
:10A54000059009380179C27808021043082802DA18
:10A550007FB046B0F0BDBF4809380179C278080223
:10A560001043BD49884217DD0022BC49BC48FFF7B3
:10A57000D1FE0021B748093841718171C170017164
:10A58000C17101720122B549B548FFF7C3FEB5A1FB
:10A590000120FFF7B5FADBE7AE4809380179C27848
:10A5A0000E0216430022AD49AD48FFF7B3FEA9489D
:10A5B00009380179C27808021043001B81B2A5480E
:10A5C0000938C170090A01710122A449A448FFF7A2
:10A5D000A1FE042E00DABBE7102E01DA354600E0BA
:10A5E00010259C480938017AC2790F0217430024CC
:10A5F0000DE00598C05D07A90855781C80B2074694
:10A600005F21C900884200DD0027601C84B2AC4293
:10A61000EFDB98A107A8FFF78BFA00286AD08D48D6
:10A620000938017AC2790F02174300240EE0059819
:10A63000C05D0A2800D10BE0781C80B207465F217C
:10A64000C900884200DB0027601C84B2B442EEDB04
:10A6500000BFB4424DDA601C85B2002421E07D4881
:10A660000938017AC279080210430599085C07A9E4
:10A67000085578480938017AC27908021043401C0D
:10A6800081B274480938C1710A0A02725F20C000A1
:10A69000814204DB00216F480938C1710172601CDE
:10A6A00084B2AC42DBDB002007A9085500226B49CD
:10A6B0006B48FFF72FFE674809380179C278080216
:10A6C0001043401B81B263480938C170090A017107
:10A6D000012262496248FFF71DFE681C81B207A88B
:10A6E000FDF79CFC002803D065A10020FFF708FAC5
:10A6F0002EE72DE7102E00DA2AE756480938017AAE
:10A70000C2790F021743002001900690002425E033
:10A710000598C05D029002982C2808D10198012864
:10A7200004DA0198401CC0B201900DE018E00198D5
:10A73000012809D10698042806DA0698421C92B22C
:10A740000299069203AA1154781C80B207465F2131
:10A75000C900884200DB0027601C84B2B442D7DB0A
:10A7600000BFB44200DBF3E6002103AA06981154AF
:10A7700003A8FAF72DFC85B20A2D02DA0120069013
:10A780000DE0642D02DA0220069008E07D20C00072
:10A79000854202DA0320069001E004200690069824
:10A7A00028180E3085B208A80079552801D1681CF8
:10A7B00085B2AE4200DACBE6002421E02548093814
:10A7C000017AC279080210430599085C07A9085567
:10A7D00020480938017AC27908021043401C81B22E
:10A7E0001C480938C1710A0A02725F20C000814208
:10A7F00004DB002117480938C1710172601C84B262
:10A80000AC42DBDB002007A908550022134914489D
:10A81000FFF780FD0F4809380179C278080210431C
:10A82000401B81B20B480938C170090A017101222D
:10A830000A490B48FFF76EFD681C81B207A8FDF7B7
:10A84000EDFB002803D012A10020FFF759F900BF4B
:10A850007EE600009D0A0020F602000005010500CA
:10A8600000440040527832427566204F7665720D82
:10A870000A0000002B5A4950524543560000000080
:10A8800051756575652046756C6C310D0A000000C8
:10A8900051756575652046756C6C320D0A000000B7
:10A8A000F0B58BB004460D4616461F4601210846FA
:10A8B000FEF76AFB002F27D02846FAF7C7FF20468D
:10A8C000283000901198019010200290C820039029
:10A8D00000200490802005900020069007900890AA
:10A8E00009900A9069462846FBF718F80122802152
:10A8F0002046FFF7D4FC012202212846FBF704F88A
:10A9000001212846FAF794FF1098002825D03046F8
:10A91000FAF79CFF20462430009012980190002006
:10A920000290C82003900020049080200590002011
:10A9300006900790089001204003099000200A909B
:10A9400069463046FAF7EAFF012240212046FFF728
:10A95000A6FC01213046FAF76BFF0BB0F0BD0000FA
:10A9600010B50120054908810022114604A0FDF719
:10A9700095F808A10020FFF7C3F810BD2004004897
:10A9800041542B504F433D31303030303031380D51
:10A990000A000000555F504F4320566572210D0A92
:10A9A0000000000010B50D4881784278080210437D
:10A9B000002800D110BD0948001DFDF773FC0021DF
:10A9C000064841708170C820054948630121044848
:10A9D0003030FAF72DFF00BFECE70000000900203F
:10A9E0000000024010B500F001F810BD00B58BB0BA
:10A9F00001218803FEF7E8FA01220921C806FBF7C6
:10AA000061FB01220A210920C006FBF75BFB032042
:10AA100040020990022108A801720321417200211D
:10AA200081720121C17209A90920C006FBF702FB4E
:10AA3000E1204002039000200490059006900890C9
:10AA40000820079003A91748FFF786FC0121154845
:10AA5000FFF719FC40211348FFF70AFC00221249B6
:10AA60001048FFF757FC00201049086210480146C3
:10AA7000C831012213460092019102900B4A3032F4
:10AA80000A491C310748FFF70BFF00210848001F47
:10AA90004170817000200649091FC87008700BB012
:10AAA00000BD00000038014007010700000002401F
:10AAB0000409002000B58BB001214804FEF774FAA8
:10AAC000012202210920C006FBF7FCFA0122032122
:10AAD0000920C006FBF7F6FA0C200990022108A80D
:10AAE000017203214172002181720121C17209A901
:10AAF0000920C006FBF79EFAE120400203900020E7
:10AB000004900590069008900C20079003A91B481C
:10AB1000FFF722FC1A481B490022012300920191F1
:10AB20000290194A184914391448FFF7B9FE002257
:10AB300040211248FFF7B3FB012214490F48FFF7E9
:10AB4000E9FB01210D48FFF79EFB40210B48FFF771
:10AB50008FFB00210A480938C17001714171817170
:10AB6000C171017200200649093988705F21C9004E
:10AB70000348FAF7C4F90BB000BD000000440040E0
:10AB80009D0A0020950D0020580002400501050097
:10AB9000F0B591B0002211461CA0FCF77FFF002504
:10ABA0002BE032260022114621A0FCF777FF1DE0A2
:10ABB00041216846FDF7AAF90446002C12D0062C64
:10ABC00014D123A16846FCF7FFFF002804D121A17E
:10ABD000FEF796FF11B0F0BD002211460BA0FCF766
:10ABE0005DFF03E00120204FBC4600DF3046711EB0
:10ABF000CEB20028DCD1681CC5B2052DD1DB1BA16B
:10AC00000020FEF77DFF00BFE4E7000061742B73B6
:10AC10007973636D643D73746172745F70636D20EA
:10AC2000766F6C756D65203720350D0A00000000C9
:10AC300061742B737973636D643D73746172745FB7
:10AC400070636D20766F6C756D650D0A00000000F5
:10AC5000372035005B30375D53657420566F6C7557
:10AC60006D65206F6B000000C5B500085B30375D77
:10AC700053657420566F6C756D65206661696C65EF
:10AC800064000000F0B589B01BA10020FEF738FF7A
:10AC9000002529E03226002211461BA0FCF7FEFE0B
:10ACA0001DE01E2101A8FDF731F90446002C12D049
:10ACB00017A101A8FCF788FF002805D015A101A85D
:10ACC000FCF782FF00280AD115A10020FEF718FF2B
:10ACD000002009B0F0BD0120154FBC4600DF304612
:10ACE000761E0028DDD16D1C642DD3DB11A1002060
:10ACF000FEF706FF0120ECE7576169744D6F64654C
:10AD00006D52756E3A0D0A00415445300D0A00002F
:10AD10004F4B00002B504F433A53544152540000C4
:10AD20004D6F64656D2052756E696E670D0A000087
:10AD3000C5B5000854696D654F75740017484078B3
:10AD4000002800D1704715480078012804D100215F
:10AD50001348C1710172F5E712480078401CC0B277
:10AD600010490870632800DAECE700200D490870EC
:10AD70000B48C079FA2805DA0948C079401CC1B2ED
:10AD80000748C1710648007AFA2805DA0448007AB3
:10AD9000401CC1B20248017200BFD3E7BC110020C1
:10ADA000DC1200206C010020F7B582B005460E468B
:10ADB000FBF7F2F83420FBF779F80120C006854252
:10ADC00002D31348854201D305B0F0BDA805800D1C
:10ADD000002800D0F8E72846FBF76EF80746042F56
:10ADE00000D0F1E700240CE0601C305C0002315D13
:10ADF000401880B2019028190199FBF7ABF8A01C0C
:10AE000084B204988442EFDBFBF79AF800BFDBE7DB
:10AE1000000001080FB410B503A9044B044A0298BE
:10AE200000F078F810BC08BC04B01847A9B30008BB
:10AE3000300100200FB41CB50A46521E019200904A
:10AE400007A9064B6A46069800F064F8009A0021AC
:10AE500011701CBC08BC04B01847000089B300087E
:10AE60000FB410B504A9074B02AA039800F052F8DA
:10AE7000044602A9002000F092FA204610BC08BC4B
:10AE800004B018479FB3000830B47446641E257898
:10AE9000641CAB4204D3635D5B00E31830BC18470D
:10AEA0001D46F8E7004870479401002002E008C8FA
:10AEB000121F08C1002AFAD170477047002001E034
:10AEC00001C1121F002AFBD1704710B5002A06DA13
:10AED00052005208D21DD308DB00102203E0D21C1E
:10AEE00093089B000C22002B02D09C188C4201D9A5
:10AEF000012010BD82188360411802604160C91AA8
:10AF0000D018884202D810600246F9E7002010608D
:10AF100010BD0000FFB591B00F460546002606E0C3
:10AF200025280AD0149A139990476D1C761C28780E
:10AF30000028F5D1304615B0F0BD00240094012161
:10AF4000F34A029400E004436D1C2B780846203B32
:10AF500098401042F7D128782A280ED0022128786C
:10AF60000246303A092A15D8009A0A235A43303A41
:10AF700080180C436D1C0090F1E701CF0090002871
:10AF800005DA01204003044300984042009002206B
:10AF900004436D1C28782E2815D1042004436878BA
:10AFA0006D1C2A280AD101CF6D1C02900BE002997A
:10AFB0000A225143303940186D1C0290287801460E
:10AFC00030390929F3D928786C2810D006DC4C28B0
:10AFD0001AD068280ED06A2817D104E0742813D03C
:10AFE0007A2812D110E00120400504430CE0012131
:10AFF000090501E0032109050C436978814203D169
:10B000000120000524186D1C6D1C287803906E2803
:10B010001ED00CDC632831D004DC00288AD05828EC
:10B0200011D1B2E064287BD069280CD178E0732874
:10B030002DD004DC6F2870D0702804D1A7E07528CB
:10B040006CD078286BD0149A13999047761C62E0E4
:10B050006002400F022807D003280AD0042838686D
:10B060000AD006603F1D56E03868F117066041605F
:10B07000F8E738680680F5E70670F3E73878694640
:10B0800008740020487404A80390012003E0386885
:10B0900003900020C0433F1D61070FD5002101E050
:10B0A0000199491C029A0191914213DA8142F7DB1E
:10B0B000019A0399895C0029F2D10BE0002101E09B
:10B0C0000199491C01918142FADB019A0399895C3B
:10B0D0000029F5D101990098139A401A0090214651
:10B0E000149B00F03BF901998019461807E003987A
:10B0F00003990078491C0391149A13999047019879
:10B10000401E0190401CF2D12146149B139A0098D6
:10B1100000F014F986196D1C09E741E033E034E0D2
:10B120000A200021049005916002410F022905D0F8
:10B1300001CFC2179446032905D007E0FF1DFF0881
:10B14000FF0003CF06E000B2C2179446042902D1E3
:10B1500040B2C1178C4600226146944506DA0A4681
:10B160000021404291418C462D2102E0210504D569
:10B170002B216A461176012103E0E10701D020214D
:10B18000F7E7019154E00A200BE0102009E01020BD
:10B19000049000210420044308200591029003E05C
:10B1A00008200021059104906002410F022905D07A
:10B1B00001CF00229446032906D006E0FF1DFF08B8
:10B1C000FF0003CF8C4603E080B2042900D1C0B257
:10B1D0000021019121072BD50399702906D0049AEB
:10B1E0001021059B4A401A4305D00EE040216A46D3
:10B1F0001176012108E06146014306D030216A46FC
:10B2000011760399517602210191049A0821059B38
:10B210004A401A430CD16146014301D1610707D569
:10B2200030216A461176012101910299491E02914D
:10B230000399582904D037A103910FA90F910DE06C
:10B2400039A1F9E76146059B049AF9F7DBFE039BF8
:10B250008C469B5C0F9A521E0F92137061460143FD
:10B26000F0D10F9807A9081A20300390600704D581
:10B27000012000048443029801E001200290039918
:10B28000884201DD401A00E0002041180290019838
:10B2900009180098401A0090E00306D42146149B38
:10B2A000139A009800F05AF886190020049008E0DC
:10B2B00006A9085C149A139990470498401C761CC0
:10B2C000049001998842F3DBE0030CD52146149BDE
:10B2D000139A009800F042F8861904E0149A30207E
:10B2E00013999047761C0299481E02900029F5DCBC
:10B2F00008E00F980F990078491C0F91149A139940
:10B300009047761C0399481E03900029F1DCFBE668
:10B31000092801003031323334353637383961622B
:10B3200063646566000000003031323334353637EF
:10B33000383941424344454600000000F8B5044610
:10B3400000251E461746880404D405E0394620200F
:10B35000B0476D1C641EF9D52846F8BDFFB50446FC
:10B36000002581B01E46C80301D5302700E0202704
:10B37000880404D505E038460399B0476D1C641E67
:10B38000F9D5284605B0F0BD4A68002A06D00A68FB
:10B39000531C0B6010704868401E486070470A6874
:10B3A000531C0B601070704713B50C4601216846A2
:10B3B000FFF7ACF800981CBD10B5002100F04EFA64
:10B3C00000F03CFA10BD000080B5FAF785F8FEF7F2
:10B3D000C3FBF9F785FC044A04490548054FBC4600
:10B3E00000DF002080BD0000F812002001000300F3
:10B3F000DD6E000861BA000802A0FFF70BFD00BF78
:10B40000FEE700000D0A5B4F535D457272000000BD
:10B4100000BFFEE7074801680748416100218161DC
:10B42000072101610548016AFF22120611430162EA
:10B43000401770479CBC000800E000E000ED00E011
:10B440007047000010B50446012C0AD100210548C0
:10B45000FEF77CFC04488078002802D101200349D3
:10B46000886110BD00480140BC1100200004004864
:10B470000146EFF31080C207D20F72B608680028A9
:10B4800001D003680B60002A00D162B6704700004B
:10B4900070B50D4600280FD00849094C884204D2E7
:10B4A00022680146104600F0F9F920684570054809
:10B4B00000F0C7F800F0CCFA70BD0000FFFF0000FC
:10B4C000700100200C1B002010B50E480C4942688A
:10B4D0000D480B680068934204D00A60CB88421E76
:10B4E0009A188A808A8880B2824208D10020086037
:10B4F000044800F0A6F80146024800F0F7F910BD34
:10B50000840100200C1B00207801002070B51B4D29
:10B51000E868002831D0A88A401EA882002626E0CC
:10B52000A068002808D0616841606068002802D0E7
:10B53000A16881606660A66010482146183800F056
:10B54000D5F9A08AA8826078042804D10C49E08A41
:10B5500009884018A0820120607025210855E06804
:10B56000E860E068002801D00561E6602661A88AED
:10B57000002802D1EC68002CD2D170BD241B002021
:10B580007801002070B504000ED00C4DA178286819
:10B590000126827891420BD900F0C6F928684670DE
:10B5A000204600F055FA70BD054800F04AF8F8E76B
:10B5B00066702146024800F099F970BD70010020C4
:10B5C0000C1B002010B50321FFF762FF10BD000027
:10B5D00010B50446008B084320836278618B062AED
:10B5E00015D0052A12D1084210D00A4602406283C3
:10B5F00088432083204600F0A1F9012060700221D9
:10B60000252001552146044800F070F910BD0A4676
:10B610008243EDD010BD00000C1B0020814202D3FC
:10B6200042688A4201D801207047EFF31082D207A6
:10B63000D20F72B603680B60016000D162B60020C1
:10B6400070470146406842684A600B780022022B2E
:10B6500005D0012B03D0032B01D042607047436813
:10B66000002B01D0996042608260704770B504463B
:10B67000154600202070012262702346A1702033FD
:10B6800019716060A060E06020612062A082E082A9
:10B690002083608358719871208D002803D104485D
:10B6A000FFF7E6FE20632946204600F00FF870BD44
:10B6B0008802002003480021016003490988C180F5
:10B6C000704700008401002098BC000830B5028D4E
:10B6D000920803D10E4A12881204920C036B920056
:10B6E0009A18530700D5121F01231B06403AD36353
:10B6F000002391631C469D005B1C54510E2BFAD312
:10B70000C3691362C2624163006B0249016030BDCC
:10B7100094BC0008A52E5AE2F8B5044640680026FD
:10B720000F46002805D06178022918D0A08900288A
:10B7300033D0A089E189884242D220898000001953
:10B74000076172B6A089401CA08162B62089401CA6
:10B7500080B22081E189884200D12681F8BD40680D
:10B76000002800D0012060702046FFF76AFF0546E0
:10B77000203046712189E86989000919086172B68B
:10B78000A089401CA08162B62089401C80B2208123
:10B79000E18988420AD1268108E02046FFF751FF5F
:10B7A0000546C069042107602520415501206870C5
:10B7B000284600F0C3F82946034800F097F8F8BD82
:10B7C0000320FFF719FEF8BD0C1B002070B51848C8
:10B7D000012102685170006800F0A6F8154C6578E8
:10B7E00013E0E800011948680278002A17D0012AFE
:10B7F0001AD000F0BFF8E0786D1C854200D100251A
:10B8000072B6A078401EA07062B6A0780028E8D179
:10B8100065700948FFF715FF00F01AF970BD098936
:10B8200089B2FFF7D5FEE6E78968FFF775FFE2E723
:10B8300070010020800600200C1B002005480178C4
:10B84000002902D001214170704701200249000700
:10B85000486070477C01002000ED00E070B50E4BA1
:10B86000DD789C1C1E4672B69A78AA4207D2521CFA
:10B8700022703278541CAC4200D10024347062B67D
:10B88000DC78944204D9D200D2189160506070BD27
:10B890000220FFF7B1FD70BD8006002010B5124AEE
:10B8A000D368002B17D013469B8A04E0002C12D0DB
:10B8B0002246A48AE318D4688B42F7D3C460D060D0
:10B8C0000261C468002C00D02061591A8182908ADC
:10B8D000401A908210BD0024C460D060C91A026171
:10B8E0009182848210BD0000241B002030B50278B4
:10B8F0000023022A03D0012A01D0032A00D1012308
:10B900008C7800E010464268002A02D09578A54263
:10B91000F8D24A604160002B04D0002A00D0916028
:10B92000886030BD0020FBE703494A68426000227E
:10B9300082604860704700000C1B002010B5016950
:10B9400000290FD0C268CA60C3680022002B07D04C
:10B950008B8A848A1B198B82C3681961C26000E0DC
:10B960008A82026110BD0222027000224260418080
:10B970007047000010B5416800290ED0FFF761FE46
:10B980000446FFF7DBFF01206070032125200155ED
:10B9900021460448FFF7AAFF10BD4188491C418099
:10B9A00010BD00000C1B002010B54168002911D00B
:10B9B000FFF747FE04460321203041712046FFF780
:10B9C000BDFF2046FFF7DEFD05480021006820305E
:10B9D000417102E04188491C4180002010BD0000F7
:10B9E0007001002010B50C464188002903D0491E83
:10B9F0004180002010BD002C07D00A4A436811681E
:10BA0000002B04D0FFF772FF07E0012010BD41605A
:10BA10001368002159601168886007212046FFF7EC
:10BA200037FDF2E77001002010B507480068C16AD1
:10BA3000006B814203D300680449884202D0012090
:10BA4000FFF7DAFC10BD000070010020A52E5AE2BD
:10BA500002494860022141707047000070010020D7
:10BA6000F7B5164600200446374A384902E08300FD
:10BA7000D450401C0B889842F9D3354838220188AD
:10BA80003448FFF722FA344801210088C90780B200
:10BA90004218324801683248FFF717FA3148082245
:10BAA000018831480068FFF710FA304FFF25FD701C
:10BAB0003C852F4A00213846FFF7D8FD2D48042148
:10BAC000017044602C480170C46004618482F86A8B
:10BAD0002030F9F7FFF829482A49076002207870DA
:10BAE0002748047044700978C170FFF7E3FD2648C9
:10BAF000016A2A0411430162C169026A5202920E6C
:10BB000092061143C161FFF785FC204900280860B7
:10BB100012DB82081E49920051180A688307DB0E67
:10BB20009D402A430A60C206D20E01219140401175
:10BB3000184A80008018016000233246019900985D
:10BB400000F068F8FEBD00000407002090BC00086B
:10BB5000ACBC00089801002094BC0008B0BC0008F0
:10BB600088020020B6BC0008D8000020D41A0020AB
:10BB700011B400080C1B0020241B002070010020C1
:10BB800080060020B4BC000800ED00E08001002029
:10BB900000E400E000E100E010B50B48012102687C
:10BBA00051700068FFF7C0FEFFF78EFC0748016880
:10BBB000491C0160FFF7AAFC00F00CF80448FFF7ED
:10BBC00040FDFFF745FF10BD700100207801002007
:10BBD0000C1B002070B50D4C2068002815D0A088E3
:10BBE0000B4E401EA0800AE0E888FFF72BFCA888D7
:10BBF000A0802868206029463068FFF70FFDA088E4
:10BC0000002802D12568002DEED170BD8C010020E6
:10BC1000D8000020FFB5080681B01E4617460C4626
:10BC2000000E00D14C1C1648FFF722FC050025D061
:10BC30002002000C2F632885EE61E1B22846019AAC
:10BC4000FFF714FD01240F480F4906E0A200121867
:10BC5000803AD26F002A04D0641C0A889442F5D935
:10BC60000024A10008188038C567EC702846FFF74B
:10BC700089FC0648006820304471204605B0F0BDBC
:10BC8000980100200407002090BC000870010020EB
:10BC900004000000C8000001050001007FA90300A6
:10BCA000000000001027000002000000EC0000006F
:10BCB000F803000010001C0068596364C8CCAAA7F0
:10BCC000A2ABA56E6A568A57F4BBFEFA26212D292F
:10BCD0000D093E3A37320A07F7F2FBF5FFF61C185A
:10BCE0001314F1FDF90C9F089A97929B959F121BD4
:10BCF000152C2823F92A2722242E67252F98FC7536
:10BD0000F8F33C3833340304050F06017A77726286
:10BD10006B83848EC4CB8782353F364F3D399C98E8
:10BD20009394424F4641818D4D49717D7996919D05
:10BD300099C3C41DCECA7F767C7873747E7B751ED2
:10BD40001A171F16111D47195DC7C2CBC5CFD1DD0C
:10BD5000D94C48C6C1CD61C9D78CFD88A1ADA9B168
:10BD6000BDB98B858F4B4586DCD8D3D4DED2DBD5ED
:10BD7000DFD643444E4AE747ACA8A3A4AEBA0DB7FA
:10BD8000B2AFA6E4EEEAE7E2E1ED0FE966616D69C4
:10BD9000BBB5BFB6ECE80BE3525C656F5853540C6F
:10BDA0005E5B555F312F9A0B0B5A2B9E0289593BD4
:10BDB0000E516CEBDAE631F654015C0162016A0166
:10BDC00070017C0182018A018E019A01A0BE0008E7
:10BDD00098BE00089CBE000890BE0008BCBE0008CB
:10BDE000B8BE0008B0BE0008B4BE0008C8BE000857
:10BDF000C0BE0008C4BE0008ACBE0008A4BE000857
:10BE0000CCBE00084B000400004040404040404091
:10BE1000404041414141414040404040404040401D
:10BE200040404040404040404005020202020202C1
:10BE30000202020202020202022020202020202010
:10BE40002020200202020202020290909090909024
:10BE500010101010101010101010101010101010E2
:10BE60001010101002020202020288888888888856
:10BE70000808080808080808080808080808080842
:10BE800008080808020202024000000009BE00087B
:10BE9000464F54410000000054470000444D00004C
:10BEA000544D00005241504E0000000041504E00E1
:10BEB00053475000524D5000534D500053545000C2
:10BEC00056455200424154005053540000000000B7
:10BED000F0BE0008C0000020D8000000ACAE000892
:10BEE000C8BF000898010020A81D0000BCAE0008D3
:10BEF0000000000000366E0100000000000000009D
:10BF000001020304060708091407002000000000CE
:10BF10000000000000000000000000000102030417
:10BF200001020304060708090000000000000000E9
:10BF3000FFFF000000FFFF00000000000000000005
:10BF400000000000000000000000000000000000F1
:10BF5000000000005500000000000000000000008C
:10BF6000000000000000FFFF0000000000000000D3
:10BF7000000000000000000064000000000000005D
:10BF8000640000000000000000000000000000004D
:10BF900000000000000000000000000000000000A1
:10BFA0000000000000000000000000000000000091
:10BFB0000000000000000000000000000000000081
:08BFC000000000000000000079
:0400000508004CC1E2
:00000001FF
